:020000041100E9
:10300000002373B52B4D2C4C28006361022601F080
:103010007DF94021FE2221742800284B009601F002
:10302000C7F9002836D1217CFF222800244B0096C6
:1030300001F0BEF900282DD1224BA2899A4226D157
:10304000E389214A93420DD1204B6361204B2268D2
:10305000002A03D1002B01D043CB43C4280001F048
:1030600093F973BD1B4A934201D00023EFE71A4B3B
:103070001A4A1B68934206D9C02304222800217CE7
:103080009B0001F00BFA114B6361154BDFE7002346
:103090002374EAE7CC233821AC2228009B01217459
:1030A00001F0FCF90028F2D10E4B63610E4BE38175
:1030B0000E4BCCE7F441FF1FA461FF1FB061FF1F5F
:1030C000B261FF1F5959000083050000394100110A
:1030D00068BD001182150000C861FF1F8713000042
:1030E00074BD0011F1410011AAAAFFFF5CBD0011DF
:1030F000F7B5164B0192C318021D002000938823D8
:103100005B05D3181B685C1C1AD09CB2402C18D8E5
:103110008D781E0CAC466746CD782D023D43AE42FD
:1031200006D1019800280ED110000C70240A4C70B2
:1031300003249BB20733A343D218009B9A42DED3E9
:10314000FEBD4432F9E71000FAE7C046FC0F00006C
:10315000802213B503000324019189B25201073183
:103160009B18A14304305A1A88235B05C3181B68B7
:10317000591C03D190429241104016BD99B240298A
:1031800007D80B000733A343C0189042ECD30020AC
:10319000F3E74430F9E7134B134A1B68126810B584
:1031A000FA24934201D81A00F824104BE4021B6859
:1031B0009A4210D813000E4A12689A420ED3013375
:1031C00007D1F823DB029C4203D10A49054808F0E5
:1031D00047FD200010BDFC24E402ECE7FE24E402DD
:1031E000F7E7C04600C0071100D0071100E0071143
:1031F00000F00711FFFFFF7FF0B59BB015000490B2
:103200000391402A00D9A0E006AB59801A80FFF74D
:10321000C2FF0400042816D9002206A9FFF768FFA0
:10322000052810D906AB1B88AB420CD1002D07D066
:10323000514B2A000499C01808F0AAFB002802D1BB
:1032400001201BB0F0BD06AB1D8020000699FFF7E2
:103250007FFF041E7BD1069B0793FFF79CFF802313
:103260005B01C618802307001B039E4201D3F8268A
:10327000F60288235B05F31801931B68013302D023
:10328000019808F0BDFB3D49019808F0E9FC3B1DA1
:103290000293331D05938822029B52059B181B68DD
:1032A00008935A1C3CD044219AB20091402A04D879
:1032B0000320D11D814389B2009103991B0C8B42DD
:1032C00024D0402A22D80122300008A9FFF710FF9D
:1032D000021E1BD1380008A9FFF70AFF04000428CA
:1032E00031D9009A059B9B1880225201B218934253
:1032F00040D288235B05C118009A09A808F000FC99
:103300001D4B009A09A9F01808F032FC009A029BA4
:103310009446634402931A4B029AFB189A42BAD31A
:1033200088235B05FC1821680198013908F098FC96
:10333000200008F065FB039A07AB5A80300007991C
:10334000FFF706FF0400002C03D1002079E70428D2
:10335000FBD988235B05E018069908F081FC03235C
:10336000EA1C9A4300D16BE7034B0499E01808F07C
:10337000FFFB65E70424ECE704000011FFFFFF7F7B
:10338000F80F0000F7B505001400402A21D80027E7
:1033900001AE71803780FFF7FEFE042816D93A008F
:1033A0003100FFF7A5FE042810D93688BC420BD0A7
:1033B000BD4209D0221CB44200D9321C064B92B245
:1033C000C118280008F09CFB30B2FEBDC04300B21B
:1033D000FBE703204042F8E70400001137B5042260
:1033E00004000D0001A81649FFF7CCFF02000428D5
:1033F0000BD1019BA34208D3AB4204D0104901A8D2
:103400000195FFF7F9FE01203EBD0E4C2368200018
:10341000019308F0F5FA019920000139019108F0B3
:103420001FFC80235B01E418074B9C42EED1042271
:10343000034901A80195FFF7DFFE0020E4E7C0463D
:103440005555000000C007110000081130B589B0C3
:1034500008F0B6F910226946254808F0A9FA254B6C
:10346000009A9A420ED1019B029A0F2B33D8002169
:1034700001240698013B08D2002900D00292029B49
:10348000013331D10023029325E0551CF2D1020013
:103490002100EFE710341022200004A908F088FA78
:1034A000029B013301D1069B0293882304995B059B
:1034B000C918059B06981A03120B049105928142C4
:1034C00003D02B4201D108F01BFB019B013B019370
:1034D000019B002BDED1029B002B03D004930498A8
:1034E0004168084709B030BDE025014C2D03EFE7E6
:1034F00000000111504859368022F8B5964C974B80
:10350000D200002120001C6008F032FA2300944A07
:1035100088331A60934B1A786A23002A00D011333B
:10352000E3620A232365904B37221B780820A363AC
:103530008E4B2118E361102323628D4B3B25636181
:10354000C823DB00A36123008C331A602823013ACF
:10355000E26320646364CA67043A211DCA672100DC
:10356000BC310D602100C03108602100C4310B6006
:1035700021000635CC310D602100083DC8310D60B9
:103580002100D0310A602200D43210602200D832EB
:10359000136022000227E032210017604222DC3152
:1035A0000A6021001B3DE4310D602100E831086014
:1035B0002100EC310B6023000521F4331960230056
:1035C000F0331A602300183290331A6023009433CA
:1035D000186023001E3A98331A60AF23DB00236083
:1035E000644BFA262363644B644DE360644BF03113
:1035F000A3642300FF31FC33B600A16021611E608B
:10360000A5627325E5656D3D6565A56596255D4AF1
:10361000AD00E264666258606766A566002709250A
:10362000A767E566584F594D606720002567E26738
:103630003A6015279C30676007001A203860200028
:10364000A0300700212038602000A83007004C4837
:1036500038602000F830066026006427A436376002
:1036600026005F3FAC3637602600033FB036376038
:103670002600C637B436376026000027B8363760D4
:1036800038269E60424E96205E64424E5A66DE6147
:10369000414E9A645E62F53EFF3E9E621E269A6728
:1036A000354A8000DE661F675F67DD651D6618624C
:1036B000DA67BE23394A5B00E250394BD8382350D1
:1036C00004302250C4225200A350C623E4205B00E1
:1036D000E1500433334AE1503349344BD16034492B
:1036E000800019503349E938FF3819503249043005
:1036F000195032493248D16132491163324951631C
:103700001900F4310860CE20304940001160304982
:10371000195019002F48F83108602F49D1658221CE
:103720002E4A89005A501A002D490832D1671A00D2
:103730002C49B432116088212B4A89005A501A0052
:103740002A49883211602A4ADA6408F049FA0120CD
:1037500007F096FFF8BDC0460004FF1F4064FF1F3E
:10376000206FFF1F3844FF1F4A0AFF1F3A0700005F
:1037700080C3C9019A020000DC0500006A1800003D
:1037800050C3000088130000F009FF1F204E000006
:103790006509FF1F68100000C409000040420F00C7
:1037A00010270000FC00FF1FC11BFF1F0000FF1FB0
:1037B000152CFF1FA52FFF1F3D2EFF1F811FFF1F71
:1037C0007126FF1F9D1FFF1F4921FF1F0D1FFF1F98
:1037D0009528FF1F7D29FF1FD918FF1FA127FF1F55
:1037E000C524FF1FD124FF1F0D1EFF1FC51EFF1F75
:1037F000851DFF1F0223F0B50124614D614E2B7022
:10380000614B91B01C70614F039333680021082015
:10381000FB7006F0FFFD082006F0F6FC002398423E
:1038200005D0FA78552A02D0332A00D09BE03360C5
:10383000042006F069FF08F023F8FFF75DFE08F0AA
:103840003FF81F2201240021514B10AE1A70514B3A
:103850001C70514B1970514B19689143163A0A4329
:103860001A60602219689143403A0A431A6008F0CE
:10387000FFF908F0F5F8C120FF21494B80001A58E4
:103880008A431A50C522920098588843BF39014391
:1038900099509858434908408021C901014380202C
:1038A00099509958C0050902090A0143995080218D
:1038B0003D48490108F04CF8032322003B4901949C
:1038C00000933B4807F0ACFE2C223A4905A808F0CB
:1038D00017F905AC61782078023406F0B5FCA642F1
:1038E000F8D1354C0020012106F0C2FD2268334B8F
:1038F00003201A40A023DB021343236080232268A5
:103900009B041343236022682D4B1A4080239B03A2
:10391000134323602B4A2C4B934200D8012007F01D
:1039200097FE07F005FF80232268DB041343236022
:10393000287807F09DFE039B1878C0B207F0E0FEE0
:1039400007F0B6FF2149042007F062FE06F0A8FE4A
:1039500000F0A8F800F0F8FD00F0A0FE00F01AFA60
:10396000002011B0F0BD00932100184A042008F097
:10397000DFF88023DB059C62FFF768FD58E7C0464F
:103980004A0AFF1F34F000403844FF1FD461FF1F74
:10399000480AFF1F490AFF1F680AFF1FBCF00040CA
:1039A00000E100E0FF00FFFF3C44FF1FC056FF1F87
:1039B0003C54FF1F80BC001114F00040FF7FF8FF53
:1039C000FFFF9FFF0080FF1F206FFF1F3B000108CC
:1039D00070B500252549264A26484D6308CA1B05AF
:1039E0001B0DED188242F9D100268022224B920550
:1039F0008B630921214B224C1E62224B1120DA6776
:103A0000214BDA688A43DA609A6820490A409A6052
:103A1000266007F015FF112008F012F98022636C70
:103A200093436364EE24E4006C43194A200C0400C1
:103A3000642390420AD8FA223300D200904205D97A
:103A4000144B0A21C01807F08BFEC3B2124A112092
:103A50001372D48007F07CFE104B1B78002B04D12E
:103A60000F4B1021187807F0C3FF70BD0000054010
:103A70008805054000060540FF01000000F00040F9
:103A80000038004004E100E03CF00040FFDFFFFFB1
:103A9000B70B000030F8FFFFBC61FF1FF663FF1F8C
:103AA000F461FF1F002210B51100112007F068FF1C
:103AB00010BD0000F8B500230926374F374C3B6294
:103AC000E3681120B343E36008F0BAF8112007F06F
:103AD000B7FE112008F07CF84023226880251343AC
:103AE000236080236268DB0213436360A3682C4A6F
:103AF0002B43A360A36802211340A3608023A26824
:103B00009B0113431022A360236C0720934323647B
:103B1000236C0F3A1343236480235B003B62226BC8
:103B2000204B1A402263626B1A406263A26B1A40F8
:103B3000A263E26B1340E363E3681B4A1340E36054
:103B400006F082FB0121072006F092FC174B1120A2
:103B50005A6C15435D6407F063FEFD21144B154A52
:103B600089005A508023C720626B5B031343636351
:103B7000E36880003343E3600F4B104A195811404B
:103B8000802212020A431A50802292051A600822EB
:103B90000B4B5A63F8BDC04600F000403CF00040BB
:103BA000FFFFDFFFEFFFEFFFFFFF7FFF0038004069
:103BB0000000FF1FD139001100E100E0FF00FFFF0E
:103BC0000000054030B503A804880B20002C0ED15E
:103BD0004968074D08784978090201430A20A9423B
:103BE00005D1012120001980024B1B7A137030BDD2
:103BF000192A0000BC61FF1FF7B5150008AA168836
:103C00004A680F4F14785278120222430A24BA42AB
:103C100014D10122DBB2019200962A0007F090FC39
:103C2000041E0BD1074B1B68002B07D068782A783D
:103C30000002104342425041013098472000FEBD2F
:103C4000022900004061FF1F30B5012503790400FF
:103C5000BFB02B4211D00A49408806F0DDFF284250
:103C60000BD0084B01A95B8D4D800B80064B0022C9
:103C70001B7A60880B7104F0AFF83FB030BDC046CE
:103C80003861FF1F6840FF1FBC61FF1F10B5054969
:103C9000054806F077FF0421044A054806F034FF82
:103CA00010BDC0463861FF1FFFFF0000ACBC001113
:103CB0006840FF1F10B5024804F010FF10BDC04659
:103CC000493C0011012303700B4B1A7A4270022207
:103CD00082709A78C270DA780271032242711A797E
:103CE00082715A79C2710C2202729A794272DB791E
:103CF00083720B207047C046BC61FF1F022310B5C2
:103D00000370013B43700533837010330371443BF0
:103D100043712A3383714433C37100230372064B0A
:103D200004001B8843720A30FFF7CCFF831D0A3062
:103D3000C0B2E37010BDC046BC61FF1F10B51420B7
:103D400007F08EFD124B14220021186007F010FEC0
:103D5000002007F065FF012007F06AFC022007F051
:103D6000F7FE032004F05EF9042006F073F9052045
:103D700003F09CFB062004F069F8072001F05CFAD0
:103D8000082006F0A1FE092001F036F810BDC0465B
:103D90004461FF1F07F084FD012007F041FE07F09A
:103DA00077FC0000094B10B50400984205D00129AA
:103DB00004D12000064906F0E5FE10BD0229FCD121
:103DC000013904F049FE0028F3D0F6E7FEFF0000B9
:103DD0006A61FF1F70B50D7A100004AA2C001688C6
:103DE00010221440154220D1002E20D10A78022A38
:103DF00018D14A68517815780E4A09022943914230
:103E000005D00D4A914209D01C800A2404E01422F6
:103E10000A491A8007F074FE200070BD0C22084980
:103E20001A80F7E71C800124F6E70824F4E70B2446
:103E3000F2E7C046F3FF0000F4FF0000C442FF1F9A
:103E40008CBD001110B504000749084806F09AFE21
:103E5000074804F083FD0020E40704D50721054A44
:103E6000054806F051FE10BD6A61FF1FFFFF00000C
:103E7000A53D0011F0BC0011AC40FF1F00B50C4B7C
:103E8000BFB01A780B4902A800F0C2FC6B4680B2A2
:103E9000D880002809D06A46074B01A91B88938067
:103EA000064B0022188803F097FF3FB000BDC046C4
:103EB0004861FF1F4961FF1F0641FF1F1042FF1F9E
:103EC00000B50C4BBFB01A780B4902A801F0CAFE2E
:103ED0006B4680B2D880002809D06A46074B01A9FA
:103EE0005B8D9380064B0022188803F075FF3FB06E
:103EF00000BDC0467261FF1F7361FF1FAC40FF1F12
:103F00001042FF1FF7B50E00377A1C0008AB1100F6
:103F10003D001A8820231D401F423CD13378022BDC
:103F20003BD173681F785B781B023B431E4FBB423B
:103F300008D01E4FBB4214D01D4DAB4221D00A25E4
:103F40002800FEBD002A2AD1142C2AD82200F068AD
:103F500007F0D6FD174B1C70012CF1D9FFF7B0FF0D
:103F6000EEE7002A1BD1202C1BD82200F06807F0B6
:103F7000C7FD114B04211C70104B187807F038FD59
:103F8000DEE7E3B20124009201940A00310007F059
:103F9000D7FA0500D4E70825D2E70125D0E70B259D
:103FA000CEE70D25CCE7C046F3FF0000F4FF00008C
:103FB000022900007261FF1F4861FF1FF461FF1FAB
:103FC000332310B5040003700A220749013007F0BB
:103FD00097FD064B0F201B681A0AE37222731A0C16
:103FE0001B0E6273A37310BDBC61FF1FE461FF1F52
:103FF00030B5012503790400BFB02B4213D00B4923
:10400000408806F009FE28420DD06A46084B02A8F7
:104010001B889380FFF7D4FF6B46D880002260880E
:1040200001A903F0D9FE3FB030BDC0466A61FF1F51
:104030000641FF1F10B5024804F050FD10BDC046F8
:10404000F13F001170B5160004AA148805AA15786E
:104050004A685078117800022A4A084380180528D7
:104060004BD807F08DFD03131E29343F0720042C85
:104070000BD80522121BAA4200D92A0022491A8015
:104080003000091907F03CFD002070BD0720112CFD
:10409000FBD81222121BAA4200D92A001B491A80FF
:1040A000EEE707200E2CF0D80F22121BAA4200D9EF
:1040B0002A0017491A80E3E70720032CE5D80422D9
:1040C000121BAA4200D92A0012491A80D8E70720F9
:1040D000032CDAD80422121BAA4200D92A000E4966
:1040E0001A80CDE70720032CCFD80422121BAA4246
:1040F00000D92A0009491A80C2E700220A201A8042
:10410000C3E7C046DCD5FFFF3BBD00119061FF1F38
:104110002BBD001126BD001121BD00111CBD0011D9
:1041200010B50D21024A034806F0EEFC10BDC04652
:1041300010BD00111C41FF1FF0B50024274E85B0B3
:104140003000B47100F0E2F8254D264BEA89297C55
:104150009A422FD10423300003AA00F057F904003B
:10416000300000F011F90123B371002C34D16B46FB
:1041700099892B68C9BA4B4329891B4A1B145B18C0
:1041800053806B46D9896B6849BA89B24B436989B8
:104190001B0C5B181548191C1BB2834200DD011C67
:1041A0000B0400D500211388918001331380200077
:1041B00005B0F0BD0227220003AB3000009700F0ED
:1041C000F7F80E230400297C0122300000976B448D
:1041D00000F0EEF80443C3E71C00E8E7F441FF1FDA
:1041E000A461FF1F83050000BC61FF1F0F270000B3
:1041F00073B5234E300000F089F8224D07236A463C
:104200003000297C00F002F904003000002C33D18A
:104210006B461B787F2B2FD800F0B6F86B46D8780A
:10422000F02302041B031A406B469B8816495BBAB5
:104230009BB21A432B68000953432A891B0C9B1815
:104240004B806B465A789B7812031B011A436B68AC
:10425000024353436A891B0C9B180C481A1C1BB25F
:10426000834200DD021C130400D500220B888A80E3
:1042700001330B80200076BD00F086F80124F9E7B9
:10428000F441FF1FA461FF1FBC61FF1F0F27000047
:1042900070B5114C237C002B0FD0382B0ED10F4D55
:1042A000280000F033F8CC23AC222800217C9B01AD
:1042B00000F0F4F8280000F067F870BD084BE289C0
:1042C0009A42FAD1054D280000F020F8002228007B
:1042D000217C00F0C5F8EDE7A461FF1FF441FF1F4A
:1042E0008305000010B5084B1A7C002A09D05B69D1
:1042F000002B06D09847041E01D0FEF781FE200057
:1043000010BD0124F9E7C046A461FF1F70B5C17953
:1043100005000C00631E9C411A4BE402E41849009E
:104320000460C9B2007906F0D9F8E97968794900E2
:104330000131C9B206F0D2F8E8790930C0B207F00D
:1043400047FC0023E36661332360AA795B3B002AC4
:104350000ED022689A43023B134323600A23E36191
:104360000733236200232363A3630133E36370BD38
:1043700022689A4302231343236046236361063372
:10438000A361EFE70050004070B50025040003680A
:10439000DD66C0790930C0B207F052FC29002079EF
:1043A00006F038F82900607906F034F870BD000096
:1043B000F8B51E0006AB1D78002304681700E366FD
:1043C000616007F0FDF901238022E3662B0027617D
:1043D0005200013B08D207F0B3FB08200A4A1168DB
:1043E000002D03D12800F8BD2261F2E7236F0342BC
:1043F00003D02369013D3370013613685B1A032B28
:10440000EED90125EEE7C0466008FF1F70B51C001D
:10441000002305681600EB66696007F0D1F90123F7
:104420008022EB6623005200013B08D207F088FB94
:1044300008200A4A1168002C03D1200070BD2A61AF
:10444000F2E72B6F034203D02B69013C3370013636
:1044500013685B1A032BEED90124EEE76008FF1FF7
:10446000002370B504681500E366616007F0A8F9E1
:104470000123E366256107F063FB8020064A800084
:104480001168636B034205D113685B1A032BF8D9DB
:10449000012070BD0020FCE76008FF1F70B51D0003
:1044A000002304681600E366616007F089F90123C0
:1044B000E36626610F33626B1A42FCD02B0A23613C
:1044C0001023626B1A42FCD0EDB2256107F038FB75
:1044D0008020074A80001168636B034205D113688E
:1044E0005B1A032BF8D9012070BD0020FCE7C04601
:1044F0006008FF1F70B51E00002305681400EB66FE
:10450000696007F05DF90123A619EB660F33B44229
:104510000ED107F015FB80200A4A800011686B6BF2
:1045200003420CD113685B1A032BF8D9012070BD2C
:1045300021782961696B1942FCD00134E7E700203A
:10454000F5E7C0466008FF1F10B5084CE368002B74
:1045500008D18022064B52021B689B186360054BF2
:104560001B68236007F034F9A06010BDE461FF1FF1
:10457000C8F00040CCF0004070B5184A936A916AC8
:104580009942FBD116498A689A421FD39A1A8B60C6
:10459000144B0126186893B2D202D20E4343424311
:1045A00000204C681B0A1B1912029B180E4C0A684B
:1045B0004B60551CA3420CD8002801D04B600A6008
:1045C0000A4A136008680A4B186070BD581E821AA8
:1045D000DDE7084A30009B182A00EAE700F00040B7
:1045E000E461FF1F140AFF1F40420F00C8F00040A3
:1045F000CCF00040C0BDF0FF70B51F4C23793F2BBD
:1046000001D93F2323711D4B22791A701878C0B24B
:1046100007F0AEF818231A491A4A0B801A4913807A
:104620000B805380A379194980200B800C21938043
:1046300001334B43164D191C0001834200D9011C64
:104640002980D1806379002B11D101336371237AE2
:10465000012B01D8022323726279237A0D48534338
:104660000A21584307F07CF80B4D286070BDA02B41
:10467000EDD9A023EAE7C046D861FF1F480AFF1F13
:104680000E42FF1FE443FF1F0C42FF1F0A42FF1FA1
:104690000842FF1F71020000C861FF1FF8B5152115
:1046A0000020FEF79BFE114C011E114D09D10C227A
:1046B000104BC1CBC1C4280007F05AF9FFF79CFF8B
:1046C000F8BD0C2220000C49FEF75CFE0C2802D03D
:1046D000084B43CB43C40C2228000849FEF752FE86
:1046E0000C28EBD00C220021E5E7C046D861FF1F63
:1046F000A461FF1F80BD0011FC0C0000F50C000040
:10470000F0B51D4C8022A544040088206946520162
:10471000400506F0D5FF902212016A4413002000E4
:1047200032C832C316C816C38023144C144FA6686F
:104730009B033343A3603B6007F032FA8823A068F1
:104740005B05C01807F05CF900258823290080224A
:10475000A0685B05C01840196944520007F008FAC8
:1047600080230135FF355B019D42EED1A6603E609E
:10477000044B9D44F0BDC046FCEFFFFF5443FF1FB8
:104780009808FF1F04100000F0B5040087B000284F
:1047900025D0684607F01CF91B4C022806D10622DA
:1047A0006946200007F0F4F8002816D06946002377
:1047B00001250F262F00E25C0133100910308740DD
:1047C00038002F00324097403A0002434A610439D2
:1047D000062BEFD16846FFF793FF07B0F0BD182214
:1047E00069460A4806F06CFF6A46A300D3580133B5
:1047F00005D01822FF21684607F0BAF8EAE701342D
:10480000062CF1D1E9E7C0466509FF1F0009001138
:10481000F0B5002504000E0085B0AA4200D186E064
:104820004B1C087801934B78897837790902194332
:10483000F3783F061B040B431F43039720706570FA
:10484000252800D196E033D8112813D807F070F846
:1048500069002501250125012501AA00B800B10044
:104860002501250125012501250125012501250118
:1048700005011F01232800D1DEE0DB2800D02EE156
:10488000042A00D8ACE01025052A05D0551F2A00BF
:104890003800711D07F034F905223100200007F0BF
:1048A0002FF92A003900601D07F02AF905353EE08E
:1048B000562859D010D8332800D19DE0552839D03A
:1048C0002628DAD19C4B2900132218001D0007F07E
:1048D0004FF8FEF795FB5CE0712800D177E0722875
:1048E00000D180E0602800D18BE0DC28C5D1022A0D
:1048F00000D875E07378BFB26370B378A370032AF1
:1049000005D0033A390092B2F01CFEF775FC102274
:104910003900E01CFEF736FDC51C002807DA607080
:104920005CE00C222000854907F0EAF80C252800FD
:1049300005B0F0BD013A824D0C2A13D8002A0AD0E6
:104940002800019907F0DCF8FFF756FE0C2228003A
:104950007C49FEF751FC29000C22601C07F0D0F8BE
:104960000D25E4E70C22EBE7754D774B2A0043CB8E
:1049700043C2E9E7013A704D0C2A11D8002A08D049
:104980000199280007F0BCF80C2228006F49FEF7B7
:1049900033FC29001322601C07F0B2F81425C6E787
:1049A0000C22EDE705226A49601C07F0A9F80625EC
:1049B000BDE712226749601C07F0A2F81325B6E78D
:1049C00008226549601C07F09BF80925AFE771785C
:1049D000F02905D8614B188801F0A0FD0225A6E753
:1049E000FF236370FAE75E4B012A03D072789A7056
:1049F0006270F3E79B78F4E72000FFF7E1FA050027
:104A000095E7013A564B574D062A10D8002A10D088
:104A1000012128005970019907F072F801F050F84F
:104A200029000622601C07F06BF807257FE70622A5
:104A3000EEE700225A70F3E7042A04D94A4D2F60AA
:104A400006F0C6FEA860FFF797FD0422039003A9B5
:104A5000601C07F055F8052569E7444D062ADFD9A3
:104A600006222800019906F093FF0028D8D00622DC
:104A70000199280007F044F806223D492800FEF776
:104A8000BBFB0123364A91780B439370C8E7012A98
:104A9000A6D07078FFF778FEA0E7012800D0ECE6FA
:104AA000931E344F132B04D87378002B09D100F0D8
:104AB00015F9314B39001D78601C6A1E07F020F88B
:104AC00035E7551E2A000199380007F019F82B49DF
:104AD000AAB23800FEF790FB00F038F9E9E7DA28CF
:104AE0001DD1042A00D87BE7082A15D9B379727939
:104AF0001B021343F27912041A43337A1B06134341
:104B00003B603B68052231002000039306F0F8FF6C
:104B10000422601D03A956E7FE236370F1E7DE2837
:104B200000D05DE7511E012A01D10025FFE6019862
:104B300000F0ACFFF9E7C046A461FF1F8CBD001177
:104B4000D861FF1FFC0C000080BD0011F50C0000B7
:104B5000B061FF1F9061FF1F5843FF1F1042FF1FEE
:104B6000D461FF1FB442FF1FE461FF1F6509FF1FEF
:104B7000ADAC0000D563FF1FD363FF1FAEDE0000A6
:104B800070477047020010B5094B0A32094C92B2C7
:104B9000DA815A8298811882207802F025FB04225B
:104BA000054B012120781A7006F022FF10BDC04687
:104BB000E242FF1F1E64FF1F1D64FF1F013870B516
:104BC000042809D806F0DCFF030928081200234B4B
:104BD0000221187806F00CFF70BD204B08211878D0
:104BE00007F006F800221E4B1A72F5E78022002417
:104BF0001B4B1A4D52001A8108211A682878DC7262
:104C000006F06EFD2100287806F0D2FF012000F0AA
:104C100075FE00F055FFDFE7104B0821187806F00D
:104C2000E7FF1048FFF76AF80F4B104A9B79002006
:104C300093800F4A13808022094B5200D8721A8148
:104C400000F05CFE00F03CFF0A4B9B78002BC3D0C9
:104C5000094A136006F03CFEBEE7C046F461FF1F40
:104C6000C861FF1F1942FF1FD861FF1FE443FF1FE8
:104C70000A42FF1FD461FF1F34F0004010B5012924
:104C80000BD1082809D1054B1B78002B05D0262213
:104C9000034B04485A72FFF775FF10BDF663FF1F00
:104CA000C861FF1FC40900000300F0B50A4D8E184B
:104CB000B14202D152008018F0BD0C782F6824094F
:104CC0003C5D0F271C700C7801313C402F683C5D27
:104CD0005C700233ECE7C0460442FF1F0E22124B09
:104CE00010B51A700D23114C11492370093A043B79
:104CF0001048637006F004FF2D2301220E490F486F
:104D0000E371FFF7D1FF01220D49FFF7CDFF01222B
:104D10000C49FFF7C9FF030000200B49020018707F
:104D2000FEF76AFA10BDC046F263FF1FD363FF1F90
:104D30003BBD0011D563FF1F6709FF1FDB63FF1F2A
:104D40006609FF1F6509FF1FAEDE000070B5124C3B
:104D5000142220001149FEF715FB431E104D132BA2
:104D600017D8AB78002B14D0431C2B7009236B7021
:104D7000002300190370287829000130C0B206F022
:104D8000C7FE297822000139C9B2002005F0DAFDFA
:104D900070BDFFF7A3FFEEE7D563FF1FAEDE000097
:104DA000D363FF1F10B5114B1A781870002A0ED06C
:104DB00000280BD10E4B1A78062A07D85423D3406B
:104DC000DB0703D50B4B187802F00EFA10BD002854
:104DD000FCD0074B1B78012B02D0033B022BF5D8EC
:104DE000044B0121187806F003FEEFE7F663FF1F7E
:104DF0001D64FF1F1E64FF1F70B5514E514A52497A
:104E00003070082005F02AFC0121022005F030FB5B
:104E1000022005F011FC0121002005F029FB0020F3
:104E200005F00AFC00F0BAFEFEF7EAF806F028FEEC
:104E3000032246494648FFF737FF2D24030004228A
:104E40001C7044490130FFF72FFF30230470424D9E
:104E5000424C437083702E3B062220004049EB8772
:104E6000FEF790FA062813D0200006F0B1FD0228C4
:104E700009D00321200006F01BFE8D23E3706E3B5A
:104E8000237119336371062220003549FEF7B4F906
:104E9000344B1B68FC335C64FFF758FF0020FFF7BE
:104EA00081FF314C314A0121314B1278207802F0D8
:104EB0005DF9304A304B12780021207802F056F923
:104EC00001222E4B1A702E4BDB78552B31D12D4BF6
:104ED0003B325A722C4B2D4AAB81EA812B826A827B
:104EE0002021307806F0C4FC0120404205F076FD18
:104EF0000120404205F012FEFFF712F9FEF7C6FE50
:104F000000F0A4FC01204042FEF79CFF012006F0C7
:104F1000BFFDF02001F0E6FA0121307806F068FDCF
:104F2000307802F0BDFA1A4806F0D2FBFEF7C2FD57
:104F300070BD6422174B5B7953431A000A32CBE7EA
:104F4000F461FF1F814B00117D4C00115843FF1F7E
:104F50009061FF1FB061FF1FE242FF1F6509FF1F45
:104F6000ADAC00004064FF1F1E64FF1F3842FF1FEE
:104F70001942FF1FF263FF1FD363FF1FC463FF1FAC
:104F8000D461FF1FC861FF1FC4090000CE090000E3
:104F9000F661FF1FD861FF1FF8B50A0020230D003E
:104FA0001A40194257D0574B1B78002B50D0FFF7AF
:104FB000E3FA554B554C564E99686268737A8A1AD3
:104FC000DB039A4202D36160FEF774FD327A217AE4
:104FD000531EDBB2994205D1FFF75AF9002000F0C9
:104FE000A5FD0FE09142F9D300232372FFF77AF970
:104FF000012000F09BFD474F3800FEF77FFE39008F
:1050000006F0DEFC637A002B1FD0013BDBB263723B
:10501000002B1AD1404BDB78552B01D106F058FC00
:10502000E37A002B0CD000233C4A3A4FE3721388FA
:10503000380001331380FEF761FE390006F0C0FC32
:10504000642370795843FFF79DFD237A013323725F
:1050500020206840F8BD0BB2002B0ADA304B1878DC
:1050600006F0CEFB002801D006F0F2FD8020000201
:10507000EFE70224214206D0244B01201A72FFF7E9
:1050800091FE2000E5E70B071ED5FFF775FA1E4BD2
:105090001E491F4C98684A68637A821ADB039A4259
:1050A00002D34860FEF706FDFFF71CF9FFF7F0F8A2
:1050B000012000F03BFD00F0E3FB2368DB0701D596
:1050C000FEF7B8FF0820C4E71024214206D00D4B9C
:1050D0001B78002BD5D1FEF7EDFDD2E7012421424C
:1050E00007D0104800F06CF806F012FB00F004FD49
:1050F000C7E70424080020402142ABD0FEF7BEFEE3
:10510000BFE7C046F663FF1FE461FF1FC861FF1FD2
:10511000D861FF1F1942FF1FD461FF1FBC61FF1F31
:10512000F461FF1FFC41FF1FF0B51B4B1B4F1B8899
:105130003A8804001A4E1B4D85B09A420DD8328829
:105140009A420AD3184B1A882B889A4205D1174ADB
:10515000174B12881B889A421BD0052001F018FAC1
:105160003B8802AA13803388019053802B88114D0D
:1051700093800F4B02A91B88D3800F4B2A78188885
:1051800002F034FF0D4B08212878019A1C7006F0BC
:1051900027FB05B0F0BDC046C263FF1F0E42FF1FD4
:1051A0000C42FF1F0A42FF1FC063FF1FBE63FF1FA9
:1051B0000842FF1F1E64FF1F1042FF1FBC63FF1F3A
:1051C00013B50C4B1C78002C11D1002801D00A4BD0
:1051D00018600A4A0A4B11780A4A10780A4A019262
:1051E0000A4A0092002205F0A5FA200016BD1124FB
:1051F000FBE7C0461D64FF1FB863FF1F1C64FF1F51
:105200000C64FF1F1E64FF1FF863FF1FFC63FF1F7A
:1052100010B5064B12201B78052B06D1044B132228
:105220001988044B187801F08FFB10BD1D64FF1F17
:105230001042FF1F1E64FF1F10B500240122114BF6
:1052400052421870104B1C70104B1A8002F028F953
:1052500004220F4B21001A700E480C3206F000FA9F
:10526000102221000C4806F0FBF907220B4B1C60B2
:105270000B4B1C700B4B1C700B4B1A700B4B1C70A8
:1052800010BDC0461E64FF1F1D64FF1F1042FF1F9C
:105290001C64FF1F0C64FF1FFC63FF1FF863FF1FEC
:1052A000D263FF1FD163FF1F1242FF1FD063FF1F96
:1052B000F8B5174C0600257806A814240078052DAB
:1052C00023D1B41F134FA5B21824BD421DD88D1F82
:1052D000ADB2BD4219D8FA256D00AA4215D21D0003
:1052E0000D4F0A3DADB2BD420FD80C4C26800C4C80
:1052F00021800C4900240A800B4A1380FFF714FF19
:105300000A4B0421187806F073FC2000F8BDC04653
:105310001D64FF1F790C0000750C00000E42FF1F7A
:105320000C42FF1F0A42FF1F0842FF1F1E64FF1F9F
:10533000F0B50BB20D0089B0002B00DB70E1A44E7C
:10534000307806F05DFA041E50D00378A22B00D10D
:1053500022E1D02B1AD0912B45D143780E2B42D18C
:105360009C4B82889A423ED19B4A83681278052AD8
:1053700039D1032018567F2835D0984B1B68002B55
:1053800031D05B68002B2ED098472CE0807807281E
:1053900029D806F0F5FB0428183F3F74A8D8637895
:1053A000002B0CD101218C4B19708D4B1A78002ADF
:1053B0005BD08C4B307801F0D9FE002855D0072205
:1053C000854B1A7051E061780029F8D1E378002B01
:1053D00011D0854A854B1278307801F0C7FE607095
:1053E0006378002BEBD1200006F032FC8020000215
:1053F000684009B0F0BD784B1B78022BF3D0012137
:10540000307806F0F5F90028EAD10121307806F06D
:10541000EFFAE5E76378002BD1D16F4F032807D16E
:105420003B78052B02D101333B701EE00223FBE7E2
:105430006F4B1A886F4B0293002A0BD01B78002BFE
:1054400003D00121307806F0CBF93B78062B04D14C
:10545000013BE9E7029B1A70F7E7042B41D10121D8
:10546000029B3078197006F0C3FA5C4B1B68002B66
:10547000B9D01B68002BB6D0574A107884E7637800
:10548000554F002B27D10622211D5B4806F038FB23
:1054900062895A4B5A491A80A2895A4B1A80E38969
:1054A0000B800521397058490A80584A1380228A96
:1054B000574B1A80574B1B78012B09D11F2001F045
:1054C00067F8FA22920042430421307806F088F906
:1054D0000022484B75E7312B00D070E70022454B86
:1054E0001A700323A0E706220021434806F0B8F80B
:1054F0000023454A04211380444A30781380444AEB
:10550000138006F075FB0821307806F071FBA37953
:10551000083B5A425341304A03331370304B1B78D7
:10552000002B06D0334B30781A78002A06D001F0D1
:105530005BFE0122314B52421A8096E7012119701D
:1055400006F056FAF5E70821307806F051FB63784B
:10555000002B00D047E72C4B2D4F0293E388029A93
:1055600004211380294B307803932389039A1380F5
:1055700063893B8006F03CF9002800D033E7264BD6
:105580001B68002B00D12EE7039902983A880988FE
:1055900000881B68984726E74379132B00D022E741
:1055A0000389012B0AD11D4B1B78022B06D1082140
:1055B000307806F01DFBFFF72BFE14E7052000F006
:1055C000E7FF08210200307806F00AF90BE7C04631
:1055D0001E64FF1F051400001D64FF1FB863FF1F3A
:1055E0003842FF1F1942FF1FF263FF1FD363FF1FE3
:1055F000F463FF1FF663FF1FC563FF1F1042FF1F09
:10560000CC63FF1FCE63FF1FC263FF1FC063FF1F7A
:10561000BE63FF1FC463FF1FB463FF1FBC63FF1F94
:105620008020C001014200D0E2E6CB0731D5324BE9
:105630001B78002B1DD0314E05AC3378052B1AD1C9
:10564000023B23702E4B21001B7823722D4B1B78BD
:1056500063722D4B187801F02DFD002809D007202A
:105660002A4B30701B68002B03D01B68002B00D026
:1056700098470120BCE60E20254B06221B782549C1
:105680002370254B1B78637002ABC01806F038FA04
:10569000D8E7022308001840194209D0174B1B789D
:1056A000052B03D11D4B188806F05AF902209FE6FE
:1056B0000424214203D0FFF737FD200098E6082399
:1056C00008001840194200D193E6154B1C78012CB4
:1056D00003D0022C0DD008208AE6124B124A13493F
:1056E00013481B881288098800880094FFF7E0FDA2
:1056F000F1E7FFF78DFDEEE7F663FF1F1D64FF1F67
:105700001242FF1FD063FF1F1E64FF1FB863FF1FFD
:10571000D263FF1F1342FF1FD163FF1F1042FF1F01
:10572000BC63FF1F0842FF1F0A42FF1F0C42FF1FFE
:105730000E42FF1F10B502A804880B20002C10D1C8
:10574000496808784978090201430C48814209D127
:10575000022119800A4B59881170DB7800205BB256
:10576000537010BD074C0A20A142FAD102211980C2
:10577000034B998811705B79F0E7C0466E2A0000F0
:10578000BC61FF1F6F2A0000F7B5150008AA168834
:105790004A680F4F14785278120222430A24BA4200
:1057A00014D10122DBB2019200962A0005F0C8FE56
:1057B000041E0BD1074B1B68002B07D068782A7892
:1057C0000002104342425041013098472000FEBD84
:1057D000022900003064FF1F30B501250379040061
:1057E000BFB02B4225D01449408805F015FA284255
:1057F0000CD0124B01A95B8D00220B8002234B8041
:105800000F4B5B888B80608802F0E6FA0D49608858
:1058100005F002FAC0070CD50B4B01A91B8800222A
:105820000B8002234B80064B9B888B80608802F0A4
:10583000D3FA3FB030BDC0462864FF1F3C42FF1F73
:10584000BC61FF1F2064FF1F9642FF1F10B5074C6D
:105850000749200005F096F92000064905F092F965
:105860000721054A054805F04FF910BDFFFF00006C
:105870002864FF1F2064FF1FACBD00113C42FF1FC6
:1058800010B5024803F02AF910BDC046D9570011DF
:1058900070B540253F2608210B4BC207D2172A407E
:1058A000DD789C7835408C432A439C70DA708207FF
:1058B00001D521439970400704D58022D9785242FE
:1058C0000A43DA7070BDC046B442FF1F13210A4B71
:1058D000DA788A43123901400A43DA700222104210
:1058E00002D0D9780A43DA70400703D51022D9785C
:1058F0000A43DA707047C046B442FF1F10B5054B2B
:10590000082419790A00A243002801D022000A4382
:105910001A7110BDB442FF1F10B5054B2024D97871
:105920000A00A243002801D022000A43DA7010BD09
:10593000B442FF1F0821F8B5324D334BAE78040056
:105940000E40AE70984204DD67232B70273B6B70CE
:10595000F8BD2E4B984203DAE0232B701A3BF6E792
:1059600000232B706B7083B21A0029485F3292B209
:10597000284F82422CD9002C03DA5B421CB204234C
:105980002B70053420B20A2105F0EAFE04B2FA2396
:105990009B009C4232DB08232A7813432B7064213E
:1059A000200005F0DDFE0A2100B206F099F809B2E8
:1059B0002A787B5C13432B700A21200005F0D0FE6F
:1059C0000A2100B206F08CF809B27B5C6A780AE022
:1059D0006970002CDBDA5B421CB204232B70F522C9
:1059E0006B78092CE8DC13436B700A21200006F069
:1059F00077F809B27B5C1E43AE70A9E7632CCEDC5E
:105A0000EDE7C046B442FF1F1B4E00001DFCFFFF28
:105A10002A080000D7BD00110823F7B5194FCD00A3
:105A20003E7904001E403E71EDB2632806DD5F330F
:105A300033433B7140231D437D71F7BD03000933A0
:105A400005DA20235B4233433B71C623F3E70E4B59
:105A5000019300280BDA0423444224B23B710A214B
:105A6000200006F03DF8019B09B25B5CE3E70928E2
:105A7000F5DD0A2105F074FE019B00B21B5C1E439C
:105A80003E71ECE7B442FF1FD7BD0011F8B50A4FD5
:105A900005003B780E00002B0CD0084C2000FEF7D0
:105AA00035FC33002A0020003978FEF723FD200062
:105AB000FEF76AFCF8BDC0463464FF1FBC42FF1FFE
:105AC00070B50A4E0A4D06223100280005F060FF2D
:105AD000002809D0074C31000622280006F010F8F3
:105AE00007212000FFF7D2FF70BDC046B442FF1F60
:105AF000AE42FF1FAD42FF1FE622202110B50A4B28
:105B00001A70203A5A701C329A70DA780A40DA70A9
:105B1000082219791140033A0A431A71B6225A71C0
:105B2000FFF7CEFF10BDC046B442FF1F70B5184B43
:105B30005C78002C2BD1002829D0164D0A21022395
:105B4000E85E05F00DFE00B2FFF7F4FE0423E85E08
:105B5000642105F005FE012100B2FFF75DFF13226D
:105B600020002B7A9A426041C0B2FFF7D5FE032095
:105B7000FFF78EFE2000FFF7A9FE074B18780538C7
:105B800043425841C0B2FFF7B9FEFFF799FF70BD1D
:105B9000D461FF1FBC61FF1F1D64FF1F70B500258E
:105BA0000A4C2000A571FEF7B1FB11233E21200015
:105BB000074AFEF79FFCA84200D13E35054B200066
:105BC0001D700123A371FEF7DFFB70BDBC42FF1FF8
:105BD000C6BD00113464FF1F0200F0B501270A485A
:105BE0000A4E51188B1A002B00DCF0BD08241578E2
:105BF0004308684038404000805B013C58406D08D5
:105C0000002CF5D10132EDE7FFFF0000E8BD0011E7
:105C1000F0B500250F269D4200DBF0BD4C5D070965
:105C200044403440A400A05801357840F3E7000018
:105C3000F0B589B06A460D000B000F271100103532
:105C40001C780133260024093E401670547002323D
:105C5000AB42F5D12023024AFFF7DAFF09B0F0BDCD
:105C6000ECBD0011F0B54E780B7889B036020C000F
:105C7000170001901E43012A61D9954B9E4200D81E
:105C800077E001339E421CD1062A17D1CA788B785F
:105C900012021A430B791B0413434A7912061A4362
:105CA0008C4B5A6100221A705A808B4A5A608B4A78
:105CB0009A608B4ADA60002009B0F0BD8822520554
:105CC000EEE7884B9E423CD182498B78002B00D076
:105CD000F6E00C2A31D10F22A3789343E278120226
:105CE00013432279120413436279120613434B6063
:105CF000E279A07912020243207A00041043627A0A
:105D000012060243CA60E27AA07A1202024376487F
:105D10004A81834208D804236E49142201980B70EB
:105D200005F0EEFE1420C7E71201D21889235B05A7
:105D30009A42F0D801238B70BDE7022AFAD00523DE
:105D4000EAE76A4A01239642E6D1FFF761FA052F96
:105D50000CD9E378A2781B021343227912041A4368
:105D600063791B061343624A0393136005F0B0FD89
:105D7000A1E7584D2B78002B9DD1AB78002B00D19B
:105D8000A0E02B8901339BB20093B34200D091E095
:105D9000132AD4D9CF7C8B7C3F02122120001F43D1
:105DA000FFF71AFF874200D08EE0002E3DD1E37846
:105DB000A2781B0213432279E96812041A4363791B
:105DC0001B06134303930A228B4212D1FF23A370B5
:105DD000E370237163716B89002B09D1E37B227C13
:105DE0001B0212041343A27B13431B0901336B8173
:105DF00000226B89002B8ED0002A67D1686837019A
:105E00003818000B6B6900030390984205D968614C
:105E100005F0F6FDEB780133EB7068681022A11CE9
:105E2000381805F0A5FE2E8145E76F89009A7B1E84
:105E30009BB293423AD1E278A37812021A432379B3
:105E400005A81B04134362796C6812061A43EB68B9
:105E500000920392211D0C22049305F051FE0120B3
:105E6000260004A940421036FFF7E2FE013F012F51
:105E700017D1009A0B232861824200D04CE70422FC
:105E80001C49200005F074FE042203A9686805F08F
:105E900017FCE968039AFF23914200D13CE7F73BE6
:105EA0003AE73100FFF7C4FE1036DFE70923B742B7
:105EB000A4D831E7009BB34200D9FCE607232BE7C7
:105EC000022329E7032327E7062325E70A2323E7FD
:105ED000FFFE0000C442FF1F00000111FFFF000091
:105EE0005048593601FF0000FFFF001102FF00007B
:105EF00034F00040D042FF1F10B5034C0B000122CC
:105F0000210000F06BFA10BDB96000110B8870B56C
:105F100006000D000224162B11D92B00032209497B
:105F200000F05CFA041E0AD1074B2A881B88191C52
:105F3000934200D9111C300089B200F0EFFA200022
:105F400070BDC046E56000115A64FF1F10B54A7865
:105F50000400013A0B000220012A07D80A78002A1F
:105F600004D005222000024900F038FA10BDC046D6
:105F7000136100110A7810B50B0004000220002AFA
:105F800004D007222000024900F028FA10BDC046C4
:105F9000BF6100110A7810B50B0004000220002A2E
:105FA00004D009222000024900F018FA10BDC046B2
:105FB0002562001110B5034C0B000B22210000F0EC
:105FC0000DFA10BD5562001110B5034C0B000D22E7
:105FD000210000F003FA10BDC762001110B5034C98
:105FE0000B000F22210000F0F9F910BD2163001110
:105FF0000A7810B50B0004000220002A04D01122F8
:106000002000024900F0EAF910BDC04631630011DA
:10601000002310B51322190000F0E0F910BD0000B4
:1060200010B5034C0B001722210000F0D7F910BD6A
:1060300083630011002310B51922190000F0CEF976
:1060400010BD000010B5034C0B001B22210000F016
:10605000C5F910BDBD630011F7B584890D000600B8
:106060000121002C22D000238268D3561778002B00
:106070001EDA0C2C1AD90C3CA4B2131940880093D8
:10608000230002F086FE431E984101307B06DB0FA1
:106090006B703F23013C1F40A4B22870AF70AC80EE
:1060A000002C07D0B3680133AB6000210800FEBDAF
:1060B0000020EBE7AC60F8E70B7803704B88437087
:1060C0004B881B0A83700B79C3700420704704202F
:1060D000022B06D10020537811781B02009A0B4343
:1060E000138070470B8803700B881B0A43700220D3
:1060F00070470420009983420AD1537810781B021C
:1061000003430B80D37890781B02034300204B801D
:106110007047F8B50D004B7801240021461C037030
:106120002B788B4201D82000F8BD6B78B01C4F1C37
:10613000012B10D1890069184B88022233704B88DB
:10614000B9001B0A7370691805F02AFB0436043481
:10615000A4B2F9B2E4E7122359436B185A88043108
:1061600032705B8810221B0A7370691805F018FBE7
:1061700012361234ECE770B5049D14001E00052B96
:1061800001D8042070BD637812781B0213432B8062
:10619000E378A2781B02134302226B802A71211D2F
:1061A000681D063E05F0FCFAB2B22A81E92AE8D859
:1061B0002800A11D0A3005F0F3FA0020E2E70023D1
:1061C00010B50A789A4201D8900010BD9A008A183A
:1061D0005488013304705488DBB2240A44709488D4
:1061E00084709288120AC2700430EAE710B5110078
:1061F000029C062B04D004201022142B01D010BDC9
:10620000022222714B7808781B0203432380CB784B
:1062100088781B02034363800431601D05F0C0FAD7
:106220000020ECE710B50C788B7804315C43E4B2C5
:1062300003702200013005F0B3FA601C10BD042089
:10624000022B06D10020537811781B02009A0B43D1
:106250001380704710B50C000A88023105F0A0FACF
:10626000208810BD70B504000D0004981100012BAA
:1062700001D8042070BD1678527812023243028091
:106280000200F13255701470E125002C00D10C355C
:10629000023B9AB24280AA42EBD80231043005F0A8
:1062A0007FFA0020E6E70420009983420AD1537860
:1062B00010781B0203430B80D37890781B020343B2
:1062C00000204B80704710B50C000A88023105F0A1
:1062D00067FA208810BD000070B501211E0004205F
:1062E000049C0E400B4218D1CB40DDB28D4214D934
:1062F0000A49DBB2098899420FD32300EE331D709F
:106300003300580011184978165C090231430133F3
:106310002152D9B28D42F4D8002070BDDC42FF1F5B
:1063200010B50C000A88023105F03AFA208810BD39
:1063300010B50C788B7804315C43E4B20370220012
:10634000013005F02DFA601C10BD10B51100029847
:10635000032B01D8042010BD14785278043B12029C
:1063600022430280CA788C781202224342809AB279
:106370008280EB2AEED80431063005F011FA0020B5
:10638000E9E710B50C000B8803700B881B0A4370FB
:106390004B8883704B881B0AC3708A88043006318F
:1063A00005F0FEF9A088043080B210BD0420012B56
:1063B00003D100201378009A1370704710B50C00B9
:1063C0000B8803700B881B0A43704A880230043123
:1063D00005F0E6F96088023080B210BDF0B589B0F2
:1063E00003931E4B029242000700D05A019102F023
:1063F00020F81325061E2DD0029B01240370019B5B
:10640000002B04D0001903999847001984B26B46F9
:106410001B7A5BB2002B0FDA1021380002F01CFB54
:106420001925002813D130003219E1B202F066FCC0
:10643000051E0CD10C34A4B2042304AA380005A90B
:1064400093800696948101F0AFFD051E02D03000C6
:1064500005F0FEF9280009B0F0BDC0465864FF1FE2
:1064600070B505000C0000280CD00020814209D036
:1064700010222000044905F093F901202B782373A2
:106480006B78637370BDC0462CBE0011F0B506007A
:106490000D0017001C0085B002291BD00020102918
:1064A00007D1022B07D0102B03D115E00020102CB0
:1064B00008D005B0F0BD69463800FFF7D1FF2A00CB
:1064C00069460BE069463000FFF7CAFF22006946C3
:1064D000380004E0022BE9D12A003900300005F031
:1064E000B7FAE6E7031CF02800D9F0230320084997
:1064F0009AB2013A0B80D317034006499B189B10B0
:106500000B80D30F04499B185B100B807047C0466B
:10651000E042FF1FDE42FF1FDC42FF1F034B1B88D0
:106520008B4202D3024B4000C1527047E042FF1F32
:106530005864FF1F014B4000185A70475864FF1FF2
:106540001722014B1A8070475864FF1F70B5050071
:106550000E2005F0E5F9041E13D0D02303700023AC
:106560000622837007494570033005F019F9064B80
:106570002100DA8A62811B7E2373044B187805F0B0
:106580008FFA70BD7464FF1F6464FF1F3043FF1FE8
:10659000262803D8024B4000C05A70470148FCE748
:1065A000E242FF1FFFFF000070B506000C00094D1E
:1065B0001C220021280005F053F8074B1E70074BE2
:1065C0001C7005F035FB0123002801D000231220A8
:1065D0002B7070BD6464FF1F3043FF1F8564FF1F75
:1065E00070B505000D4C0800E260A160102200218A
:1065F000656005F075F9012803D11021A06802F04B
:1066000058FD10220021280005F06AF9012803D165
:106610001021606802F04DFD70BDC0466464FF1F2C
:1066200070B5041E05D1002903D006220D4805F0DF
:10663000B7F80D4B1D78012D11D1002C05D1022288
:106640001A7005F03DFA280070BD00221A70074B41
:106650001B78FF2BF7D02000FFF778FFF3E700252A
:10666000F1E7C0467464FF1F6464FF1F3043FF1FDF
:10667000030010B5002801D1002010BD00780B4A9E
:10668000002803D15988D1821B7913761378022B05
:10669000F2D10023984200D103331370044B1B78CE
:1066A000FF2B01D0FFF752FF0120E6E76464FF1FD4
:1066B0003043FF1F002911D000280CD04B7901284E
:1066C00003D140225242134303E03F2213400328E8
:1066D00002D001204B7170474022F4E70800FAE72E
:1066E00070B5094D0100287800280BD0074C062210
:1066F000200005F055F821002878FFF7DBFF200087
:1067000005F046F870BDC0468464FF1F5E64FF1F3D
:1067100000290AD0012808D13F224B799343C02B8E
:1067200003D0403B5A425341981C704770B5174DF7
:1067300006002B78FF2B15D00A2005F0F1F8041E77
:1067400010D0D0230370C83B8370114B11491B78C4
:106750004670C3700622043005F022F82100287824
:1067600005F09EF90C4B1B78012B0DD10B4B1B68D0
:10677000002B03D09B68002B00D09847084B0421C6
:106780001878084A04F0ACFF70BDC0463043FF1FC4
:106790008464FF1F5E64FF1F8064FF1FAC64FF1FE3
:1067A000B064FF1F60EA0000014B98687047C04664
:1067B0006464FF1F014BDB68186870476464FF1F47
:1067C000074B10B5DA68136801331360054B18786E
:1067D000FF2803D08021C90105F00AF910BDC04689
:1067E0006464FF1F3043FF1FF7B50E0002F0C8F8C6
:1067F000051E1CD00E4B06621F78002F00D10778B3
:10680000AB791020019305F08BF8041E0FD0D02334
:106810000380C73B8370019BE91DC37006220430CF
:1068200004F0BEFF21003800E66005F039F9F7BD3D
:106830002E43FF1F014B18787047C0468464FF1F2A
:10684000054B002805D1054B1A78054B002A00D1CD
:10685000014B18007047C0467464FF1F8464FF1F1B
:106860005E64FF1F014B58687047C0466464FF1F99
:10687000024B1868431E9841C0B270478864FF1FDE
:10688000421E03000120152A03D9FF3B5A425341FF
:10689000D8B27047F0B51C0000230E0085B00390FD
:1068A00002920B70029A934201D3002019E0E55C3A
:1068B0005A1CD2B2002DF8D0029851198142F4DC52
:1068C0000233DFB2A35C18000193FFF7D9FF002861
:1068D00007D0013D019A0399EBB233708A4202D18D
:1068E000E01905B0F0BDDB19DBB2DBE710B50C0039
:1068F00002F09EF803001220002B03D021005888DC
:1069000005F06EF810BD000070B50E4D840063599F
:10691000002B15D0186A002801D005F071F92B5909
:10692000586A002801D005F06BF92B59986A0028A5
:1069300001D005F065F9285905F062F900232B51C3
:1069400070BDC0469464FF1F1C4B70B504000E0060
:10695000150099420AD11A4B1B68002B01D1122055
:1069600070BD1B68002BFAD09847F9E7154B994288
:1069700015D1134B1B68002B0AD01B68002B07D0C6
:106980009847002804D1104B1C70104B1D70E7E78E
:1069900029002000FFF7AAFF0028E1D1F3E7080053
:1069A00001F0EEFF0028DAD003780320A342D7D10C
:1069B0002900300005F014F8D2E7C046FEFF0000C1
:1069C0009064FF1FFFFF00008D64FF1F8C64FF1F9A
:1069D000F7B50400808801F0D3FF0025A84203D05A
:1069E0000578A08802F008F81C4E3378002B1FD0E1
:1069F000AB421DD11A4B28001978FFF777FF00280A
:106A000018D000233370A3790820A778A6880193B3
:106A100004F086FF011E0DD0D0230370CA3B8370A3
:106A2000019B477086808371280005F039F801E0EA
:106A3000002DE8D1A0880B4B8200D358002B01D049
:106A4000FFF762FF1721A088FFF768FDA08801F01B
:106A500027FDA08801F0FEFDF7BDC0468D64FF1F35
:106A60008C64FF1F9464FF1FF0B587B01D000CAB52
:106A70001B88070001930DAB1B88142002930EABFB
:106A80001B88160003930FAB1B880091049310AB77
:106A90001B88059304F044FF041E1AD0D023037012
:106AA000CB3B47708370C670062229000430002D4E
:106AB00011D004F075FE019B21006381029B0098B8
:106AC000A381039BE381049B2382059BA37404F0B1
:106AD000E7FF07B0F0BD04F0C3FDECE7F7B50093A6
:106AE00008AB1B8807000C200D001600019304F072
:106AF00017FF041E13D0280001F042FF00280FD01A
:106B00000078D0232370C93BA370009B2100238110
:106B1000019B6770A580E680638104F0C1FFF7BD2B
:106B2000014B1878EDE7C0463043FF1F13B5040052
:106B300064890389C2888188C0780094FFF7CEFFFA
:106B400013BD000010B5044C2068002803D005F0E8
:106B500057F80023236010BD9864FF1FA122F0B5F1
:106B6000818892004A43384B384F1B6804009B18B9
:106B70009D2292009B18827989B01A603B68002B95
:106B80005FD01D78324B1B68002B04D05B68002B54
:106B900001D000209847260008363100E079FFF741
:106BA000B7FD237DE0710200E0780493638A290039
:106BB0000393238A0293E3890193A388009333000C
:106BC000FFF752FFE378002B0BD1E289A379A1886C
:106BD00002920196E27928000092012201F0DAFE89
:106BE000E0703B68002B20D0FFF7ACFF194D2878F0
:106BF00000281AD0184B1978FFF778FE002814D017
:106C00002B78E67808200793A78804F089FE011EF8
:106C100009D0D0230370CA3B467083708780867189
:106C2000079804F03DFF00232B701721A088FFF781
:106C300075FCA08801F034FCA08801F00BFD09B0C0
:106C4000F0BD064B9DE7C0463409FF1F9864FF1F47
:106C5000AC64FF1F8D64FF1F8C64FF1F3043FF1F58
:106C6000F8B5070008000E0001F08AFE041E18D0D7
:106C70002620FFF78DFC051E00D12578062004F0A4
:106C80004FFE041E0DD00021062204F0E9FCD023A3
:106C90002370C23B21006770A370A680E8B204F0A5
:106CA000FFFEF8BDF0B585B001930AAB1B78070075
:106CB00002930BAB1B7808000D000092039301F0C8
:106CC0005FFE061E22D0102004F02AFE041E1DD0F6
:106CD0001022002104F0C4FC2620FFF759FC0028F4
:106CE00000D13078D0232370C13BA370009B2100DA
:106CF0002372019B67706372029BA580A372039B42
:106D0000C0B2E3720C9BE36004F0CAFE05B0F0BDB4
:106D1000F7B50D00019001F033FE071E20D00E20C4
:106D200004F0FEFD041E1BD02620FFF731FC061EDA
:106D300000D13E78D0232380C53B0622A370F91DE5
:106D4000E01C04F02DFD019B2A0063810123DD403E
:106D50001A401D40210022736573F0B204F0A0FEBA
:106D6000F7BD0000F0B585B0029010000D001700CF
:106D70000A9E039301F004FE041E31D0029B002BF7
:106D80002ED1039B02795B0724D5122313430422DF
:106D9000002E08D10B99002905D10C99002902D1A8
:106DA0000D9900291AD01A430D9B2271002B00D097
:106DB000C9E0002E00D1CFE0002D00D0CCE0606A09
:106DC000002801D004F01CFF1C21300004F0B8FCA6
:106DD000606205E002239A430E33D7E793432371A1
:106DE000654BBA00D458002C00D1AAE0002E10D078
:106DF000236A002B03D11C2004F032FD20625E4B7D
:106E0000BA00D358186A002803D01C22310004F0BD
:106E1000C7FC0C9B002B12D0574CBB001D596B6A52
:106E2000002B03D1162004F01BFD6862BB00E35861
:106E3000586A002803D016220C9904F0B1FC0D9B6F
:106E4000002B11D04C4DBC006659B36A002B03D106
:106E5000142004F005FDB0622B59986A002803D075
:106E600014220D9904F09CFC380001F089FD051EE8
:106E700067D0414BBA00D358002B62D01A6A342035
:106E8000002A00D11C389A6A002A01D0143080B23E
:106E90000B9A002A01D01C3080B25B6A002B01D013
:106EA000163080B204F03CFD041E4AD018220021A6
:106EB00004F0D6FB2620FFF76BFB0190002801D1E0
:106EC0002B780193D0232370029B200063700A2348
:106ED000294EA370039BBD00A371AB59A780196A0B
:106EE0001830002905D01C22A06004F059FC2000B5
:106EF00034307359996A002907D0030014221433DF
:106F0000E060029304F04CFC02980B9B002B08D02D
:106F100003001C221C330B992061029304F040FCF7
:106F200002987359596A002903D01622606104F04F
:106F300037FC6B462100187904F0B2FD3800FFF7EA
:106F4000E3FC05B0F0BD10220D9B0D991B69A01844
:106F5000236204F025FC2CE70B9B002B00D13FE7BC
:106F6000012D00D03CE7606A002801D004F048FE03
:106F70001C210B982AE7C0469464FF1F10B5044CEF
:106F80002068002803D004F03BFE0023236010BDDE
:106F90008864FF1F0B4B07B51A68002A01D1002037
:106FA0000EBD6946531C012012780731FFF772FCB1
:106FB0000028F4D002780123100018401A42EED0C5
:106FC000EEE7C046A464FF1FF0B51F4F01203B68E9
:106FD00087B0002B25D09B78059300F0B3FB0028E9
:106FE00021D00A20FFF7D4FA04000B20FFF7D0FAD3
:106FF000164B05001E78731E9E413B68F6B2191DA4
:10700000D878FFF757FB3B682900DA7A04330392FC
:107010009A7901930292009033002000059A04F0BF
:107020009FFD07B0F0BDFFF7B5FF002805D0062093
:10703000FFF7AEFA04000720D8E70820FFF7A8FA08
:1070400004000920D2E7C0468864FF1F8464FF1F44
:1070500070B50A4E040033780D00FF2B0DD00420CC
:1070600004F05EFC011E08D0D0230370CE3B4570B7
:107070008370C470307804F013FD70BD4043FF1F6F
:1070800070B5040006200D0004F04AFC011E0AD071
:10709000D0230370CD3B8370054B44701B68858003
:1070A000187804F0FDFC002C01D0FFF767FF70BDDD
:1070B0008864FF1FF8B5264F06003B680D001124B9
:1070C000002B05D10522234B1B78134202D1122439
:1070D0002000F8BD204A10241268002AF8D0127847
:1070E000002AF5D0DB0719D52B789A1E012A1AD869
:1070F0000C2004F0B5FB132438600028E8D00023EE
:107100000A22437029000670023004F049FBFFF7A1
:107110005BFF041E0AD0FFF731FFD9E700F012FB36
:107120000028E1D1E4E7002BE2D0D0E70B4B1B783D
:10713000032BCDD11D20FFF72BFA094B1880002817
:10714000C6D0084B04211878074A04F0C9FABFE7F3
:107150008864FF1F8564FF1FA464FF1F8464FF1FF2
:107160008264FF1FB064FF1F60EA0000F7B501935F
:10717000194B14001A78052306000F0012201A423A
:1071800021D0012920D1154B1D68002D1BD00220D4
:107190001F2C18D8002C02D0019B002B13D0104BB1
:1071A0001F221E706E1C0021300004F059FA019954
:1071B0002200300004F0F4FA310020002C70002F7F
:1071C00006D004F0ADFAFEBD064B12201D68DCE7C8
:1071D00004F09EFCF7E7C0468564FF1FA464FF1F10
:1071E0004043FF1FA064FF1FF8B50F4E1224336801
:1071F000002B17D01B780F3C834213D100250B4F77
:107200000221387804F0F4FC094B042138781D8001
:1072100004F0EEFC074B28001D8033685C7004F01E
:1072200067FC04002000F8BD8864FF1FB064FF1FE6
:107230009C64FF1F8264FF1F70B5012823D11B4C83
:107240002388002B03D01A4A1578002D07D0194B3C
:107250001B68002B02D01878FFF7C6FF70BD3B2BD0
:1072600002D93C3B2380F9E7134E0221307804F029
:10727000BFFCFA222388920002215A43307804F09E
:10728000AFFA2580EAE70B4B1B68002BE6D00B4BCF
:107290001B785B07E2D5084B0221187804F0A8FCA4
:1072A0000022024B1A80FFF769FED7E79C64FF1F9C
:1072B0008064FF1F8864FF1FB064FF1F8564FF1F89
:1072C000F8B51E4D2868002803D004F099FC00236F
:1072D0002B601B4E3068002803D004F091FC002383
:1072E0003360184F05243B7818002040234221D0FA
:1072F000154800F02BFA3B78234213D0202004F0ED
:10730000AFFA2860002813D02022002104F0A8F949
:10731000202004F0A5FA041E306005D020220021B0
:1073200004F09EF9002004E0286804F069FC2C6059
:107330001320F8BD00F00AFAF4E7C046A464FF1F6A
:10734000A064FF1F8564FF1F3443FF1F10B50A4C64
:1073500023681A1E0ED0002808D10130587004F09E
:10736000C7FB002805D02368002B02D00021FFF7BF
:1073700087FE0122100010BD8864FF1FF7B5274E5D
:10738000050033680191181E21D05C78244F012C30
:1073900030D1FFF7FFFD002825D02000FFF7F8F8D7
:1073A0000400412814D91F4B022118781E4A04F00A
:1073B00097F91E4B3C3C1C80022233685A703B7884
:1073C000002B14D128000199FFF75AFE0120FEBDC1
:1073D000FA2292004243002AEED0124B0221187882
:1073E00004F0FEF9E8E7FFF7D3F80200F3E7002323
:1073F0003B70EBE73B78002BE8D1032004F090FAD8
:10740000011E08D0D0230370CC3B457083703368D5
:10741000187804F045FBFFF7B1FDD7E78864FF1F3C
:107420008064FF1FB064FF1F60EA00009C64FF1FC0
:1074300010B51749838802008B4220D011D8154916
:107440008B4217D0144900205B1899B2012907D844
:10745000926811785A425341D8B2FFF7F9FD0120E2
:1074600010BD0E4A00209B1807229BB29A42404151
:10747000C0B2F5E783681878FFF768FFF0E7836824
:1074800099785A78090218781143FFF777FFE7E7F0
:107490000A20000006200000F8DFFFFFAFDFFFFF3B
:1074A000014B18707047C0464143FF1F10B5064C92
:1074B000207001F041FA207804F0EAF905212078E3
:1074C00000F062FD10BDC046B064FF1F0BB273B583
:1074D0000D00002B00DBC4E0884B187804F090F915
:1074E000041E0ED00378912B0FD0A22B00D1A1E067
:1074F000834B1878FF2852D0210004F0D1FA0028DD
:107500004DD180200002684076BD43780F2B76D0A5
:1075100013D8052B70D00E2BEAD18088794B984276
:107520002BD8794B98421BD8784B9842E0D1A3686E
:107530001878591CFFF774F838E03E2BD8D18378BF
:10754000032B74D06CD8012B6ED0022BD0D1704B92
:107550001B68002B23D05B68002B20D098471EE0CF
:107560006C4BC0180C28C3D804F06AF81DC2C215B1
:107570000BC20B0B0B3223C23C00674BC018072811
:10758000B6D8664B1B68002B09D01B68002B06D0B1
:10759000200098470AE0A3681878FFF7C7F8200092
:1075A00004F056FBADE7A068FFF762F800289FD013
:1075B000F5E7A3681B78002BF1D0554B1B68002B17
:1075C000EDD01B68002BEAD0210055489847EDE725
:1075D0004F4B1B68002BE2D01B68002BDFD0210033
:1075E0005048F3E7504B1B68002BD8D05B68002B4A
:1075F000D5D021004348E9E7FFF7EAF9CFE78088D3
:107600004A4B984203D04A4B984200D070E7464B11
:107610001B68002BC3D05B68002BC0D02100D5E7CE
:10762000153B012BBBD963E7FFF798FAB7E7FFF7E4
:107630007DFAB4E73F4B1B78042B07D100236A4641
:1076400013800179408800F0C5FCA8E7364B1B6821
:10765000002BA4D05B68002BA1D0010036489847CE
:107660009DE7012421420AD0294B1B68002B04D03E
:107670005B68002B01D000209847012043E78B076F
:107680000AD5264B1B68002B04D05B68002B01D069
:1076900020009847022036E70421280008400D42C8
:1076A00000D131E7254E3388002B21D0013B9BB21E
:1076B0003380002B1AD1FFF7DBF800280AD0204BCB
:1076C0001C70164B1B68002B04D05B68002B01D08C
:1076D00020009847FFF7C6F8694601F001FD6846AB
:1076E000FEF7FEFF1D20FEF753FF308004200AE75F
:1076F000024B187804F07CFAF8E7C046B064FF1F2C
:107700004143FF1F0E20000001200000091000006F
:10771000A864FF1FFEDFFFFFAFDFFFFFAC64FF1FAA
:107720000C2000000B2000009064FF1F0D200000C3
:10773000132000008564FF1FFFFF00008264FF1F0D
:107740008064FF1F10B501F09BF910BD014B18605C
:107750007047C046AC64FF1F0B880020162B01D871
:1077600017230420014A13807047C0465A64FF1F44
:1077700000207047074A03001188814207D0918892
:107780000020994202D1013080001018704700207B
:10779000FAE7C046B864FF1FF0B58F7806000D0009
:1077A000C5B01E2F15D1FFF7E5FF051E03D100243C
:1077B000200045B0F0BD00223B003100C0780092AF
:1077C00000F0B2FB0400A81C00F0D2FBFF23EB701A
:1077D000EEE7264B062403931B78FF2BE8D0182FE7
:1077E000E6D87B08224A013BDB0002929A58944675
:1077F000002ADDD0029AD3185B68002BD8D0087815
:10780000002802D14B78012B02D10624122FCFD1B0
:1078100007AFAB88697800976446AA68A047041E42
:10782000C6D1AB78029A5B08013BDB00D318390064
:1078300030005B689847041E0BD1AB78042BB6D0A0
:10784000039A310010782200009700F06DFB0400CD
:10785000AEE76A78002AABD1AA7805A93B880871FF
:1078600030000A704B80FEF747FBA0E74443FF1F40
:107870003CBE00111D4B37B5050098420BD00029C6
:107880000AD1FFF777FF002805D11948FFF772FFEB
:10789000002800D0058037BD01291AD1FFF76AFF03
:1078A000041EF8D001235B420380A378FF2BF2D0A3
:1078B000FE2B07D00023E0781422009329001E330A
:1078C00000F032FBA01C00F053FB01235B426380FD
:1078D000E1E70229DFD1013901F0BEF80028DAD151
:1078E0002800FFF747FF041EDFD1D4E7FEFF0000AA
:1078F000FFFF0000022210B5074B52421A800748D2
:1079000001325A809A80DA8000F07EFA044801F051
:1079100025F8002010BDC046B864FF1F99770011FC
:10792000757800110388F7B50400002B02D10225F9
:107930002800FEBD42680221137825485268FEF7F0
:10794000A5FD00282ED0234F01253A88002AEFD02C
:10795000802321885B0201259B1A9942E8DC0C20D8
:1079600003F07EFF061E31D03B8822889C46002310
:107970001800019561469DB2491989B2AA421BD8E7
:10798000002801D062443A8000233000082208C059
:10799000210003F005FF104A1368002B13D10025C6
:1079A0001660C5E76268022113780C485268FEF73A
:1079B0006DFD0028C7D1BAE760681D0140194181FB
:1079C00001330198D6E71A001B68E6E71325AFE7F5
:1079D000AABE00114243FF1FB464FF1FA8BE0011DE
:1079E000014B18707047C0464443FF1F14230A0020
:1079F00010B51A40194204D00122102101F048F8B4
:107A000010BD4B06F9D4012088434000F8E710B5BB
:107A100014008B0604D50122102101F039F810BDA5
:107A200008230A001A40194202D14BB2002B0FDA88
:107A3000102101F02DF8002808D02300F2331B7824
:107A4000002BECD0F1342378012BE8D10020E6E7BD
:107A500003208907FAD4E2E7F0B51F00184B85B080
:107A60001C68019002910392002C27D1200005B0E0
:107A7000F0BDA5683301ED186B89019A934211D3CB
:107A8000029A93420ED8002F04D10A9B002B10D1EA
:107A90002C00EBE73B002978039A6868FEF7F6FCB8
:107AA0000028F2D10136B6B2A388B342E1D82468E7
:107AB000DAE7A3680A9A5B891380E9E70026F3E70F
:107AC000B464FF1F37B50C000A884988012391422E
:107AD00017D3002A15D0651D23792A0002210A48F0
:107AE000FEF7D4FC102300280BD02379618820886E
:107AF00000242A000094FFF7AFFF0A23A04200D021
:107B0000230018003EBDC046AABE001113B50A00EE
:107B100008884988012388420BD8002809D000240E
:107B2000137905320094FFF797FF0A23A04200D093
:107B30002300180016BD13B50A00088849880123E0
:107B400088420BD8002809D000241379053200940C
:107B5000FFF782FF0A23A04200D02300180016BDC1
:107B6000F0B58BB003904A8808880E00012382424A
:107B700055D3002853D00023012704AC23700022E2
:107B8000718813000092FFF767FF051E3ED0207832
:107B9000002835D12B78022B18D167706A898300B1
:107BA0000130E31880005A8069680222201803F02F
:107BB000F7FD23780133DBB22370042B19D93B0086
:107BC0006889013080B2002BD9D01FE00223637096
:107BD000122358436A89231804305A806968102296
:107BE000201803F0DDFD23780133DBB22370002B76
:107BF000E5D10C4A6B899B185A425341DBB2DFE74F
:107C00006378012BE4D12B78022BC7D022780A238A
:107C1000002A04D021000398FEF798F900231800E9
:107C20000BB0F0BD0100FFFF0F4BF0B5040018686A
:107C3000002816D083685D89A54207D88288AE18CF
:107C4000B44203DA12019A18934201D10068EFE7B7
:107C50001E005F891036A74204D1002900D00D8094
:107C60001800F0BD3300EFE7B464FF1F70B50500E6
:107C70000C0008880021FFF7D7FF03000120002B2C
:107C800004D022002800197AFFF7C1FE70BDF7B5B5
:107C90000C00002501902300EE331B78AB4201D885
:107CA00000200AE06B00E65A00213000E718FFF7D9
:107CB000BBFF002802D126800130FEBD017A019869
:107CC000FFF794FE002802D03B882380F5E70135BA
:107CD000EDB2E0E710B5040008880021FFF7A4FF2B
:107CE00003000120002B03D02000197AFFF77EFE4D
:107CF00010BD0000054B1B68002B01D1180004E0EB
:107D00009A6852898242F6D198887047B464FF1FFE
:107D1000F0B50E27002687B0039302ABFF183E8014
:107D200005001F4B40891400984207D02B78013082
:107D300000976A6880B2FFF78FFE060002212B7859
:107D400018486A68FEF7A2FB00280FD06C89200053
:107D5000FFF7D0FF002802D0013C0419A4B2039B16
:107D6000002B00D01C80300007B0F0BD02212B7822
:107D70000D486A68FEF78AFB0028E7D102212B78BC
:107D80000A486A68FEF782FB002807D0002EDED082
:107D90003B88A342DBD17489013CDFE76C89DEE7D5
:107DA000FFFF0000AABE0011A8BE0011A6BE001170
:107DB00010B50C00FFF7DEFC03000220002B0AD0F8
:107DC000002C00D023609B781720FE2B03D00138B5
:107DD000FF2B00D1002010BD73B50D0001A90400D8
:107DE0001600FFF7E5FF172805D0002E04D1290063
:107DF0002000FEF727F976BD01221021200000F0B7
:107E000047FE0028F3D0F6E7014B18607047C046E4
:107E1000C464FF1F37B56B469D1D0100040002229C
:107E2000280003F06DFE2B88B02B0ED12379122B86
:107E300009D12300FA331B78012B06D10121608878
:107E400000F0E0F801E01B2BF8D037BD10B5054B72
:107E50000421187000F098F8FFF74CFDFEF770FB56
:107E600010BDC046C864FF1F0020F0B50BB20F0064
:107E700087B0834234DA274B187803F0C1FC051E23
:107E80002BD00378A02B25D103AE3100FEF7E4F808
:107E9000041E0BD1B378DB0724D51F4B06341B68B7
:107EA000002B03D03100688898470400A868002898
:107EB00001D003F0CDFC002C08D1184A039B1340DD
:107EC000174A934206D0B3781B2B03D00121688850
:107ED00000F098F8280003F0BBFE802000027840F4
:107EE00007B0F0BD0F4B1B68002B10D03100688825
:107EF0009847041EDAD07378002BD7D1B27801A945
:107F00000A704B800C716888FDF7F6FFCEE70624F7
:107F1000F1E7C046C864FF1FC064FF1F00FFFF00F9
:107F200000011200C464FF1FF7B50190FC200D0092
:107F300017001E0003F0F4FC04001320002C12D0E4
:107F4000B02320002370089BF4226770658026719F
:107F50000830002B08D0190003F022FC2100019802
:107F600003F09EFD0020FEBD089903F079FBF5E7C4
:107F700010B5041E06D00078FD2803D803F0C8FC15
:107F8000FF23237010BD00000A1F93B210B5040038
:107F90000220032B05D882400020024BD1529B18AF
:107FA0009C7010BDE864FF1F0B8870B5043B040093
:107FB0000D000220032B0BD80121200000F04CFD06
:107FC00003001420002B03D02900200000F0DEFB6A
:107FD00070BD000007B51300034A00920A0001219A
:107FE00000F02CFC0EBDC0461182001107B50192B5
:107FF00003220092024B0A00122100F049FC0EBD40
:108000008F82001107B56B4601AA11800449D88000
:1080100008780633012802D1190003F009FD07BDD5
:10802000C964FF1F0C4B10B518700023FF210B4AC9
:108030001380138193819380094A53801370517286
:1080400093819372D174D3821375517703F058FCE6
:1080500000F0FCF910BDC046F864FF1FE864FF1F84
:10806000CA64FF1FF0B58DB06B46002003910C224F
:108070009B5E834200DBB0E05D4B187803F0C0FBF1
:10808000051E00D1A4E00378902B00D09DE006AF40
:1080900001004688380000F013FA796804000029CE
:1080A00000D19CE03B88052B6ED13B89032B1CD96A
:1080B00005AC200000F0A2F86288172A61D839893F
:1080C000131D994231D17968237804310291D9077F
:1080D00038D5607800F08EF9071E06D000230371B2
:1080E0002378012B08D0132B23D0A868002800D1B7
:1080F00078E003F0ADFB75E06288029909A800F012
:10810000A6F80290380000F08BF909AA2378387A93
:108110000192002231000092029A00F012F9380018
:1081200000F064F9029B002BDFD0300000F080F9F2
:10813000DBE70378032BD8D16288029909A800F005
:10814000D6F8DEE7122B13D1029909A800F0B5F892
:10815000021EEAD127498B88002BC6D0887909A94D
:108160002378019161780091310000F0EAF8BCE7D2
:10817000002302AA93833000617809AAFFF72AFF3F
:10818000B3E71D4B0993F6E7042B02D09A1F012A8F
:10819000ABD8184A043B9B00995A0029A5D0D218A5
:1081A000907831003A0000F0AEF800289DD13B886D
:1081B000042B03D001213000FFF724FF012C04D150
:1081C000A868002801D003F043FB280003F040FD1D
:1081D0008020039B0002434018000DB0F0BD012831
:1081E00000D182E701213000FFF70CFFEDE7C04628
:1081F000F864FF1FE864FF1F010017000B7803708D
:108200004B784370CB788A781B02134343807047C6
:108210000A88030002700A88120A42700A88012A3A
:1082200006D14A8882704A88120AC27004207047B8
:1082300002208242FBD14A8804309A704A88120A8E
:10824000DA708A881A718A88120A5A71EFE710B5B3
:108250000400012082420CD94B780A781B02134398
:108260002380834206D1CB788A781B021343638034
:10827000002010BD022BFBD1CB788A781B02134360
:1082800063804B790A791B021343A380F0E70B88C4
:1082900003700B881B0A43704B8883704B881B0A42
:1082A000C3708B8803718B881B0A4371CB888371E1
:1082B000CB881B0AC3710820704703000120082ADD
:1082C00014D14A780878120202431A80CA78887852
:1082D000120202435A804A790879120202439A80B4
:1082E000CA798879120202430020DA80704710B5FB
:1082F00004000120022A05D100204B780A781B02D5
:108300001343238010BDF8B5060010200F001500A0
:1083100003F006FB04000120002C0ED0A0230C2249
:10832000290023806780201D002D07D003F038FA34
:108330002100300003F0B4FB0020F8BD03F090F9F9
:10834000F6E7F7B51E00009008AB142017001D7863
:10835000019103F0E5FA041E12D0A2230370019BE1
:1083600047704380099B057146710C220830002B31
:1083700007D0190003F014FA2100009803F090FBD5
:10838000F7BD099903F06CF9F6E737B5041E0FD075
:108390004388002B0CD00025C1881323007A1722B4
:1083A00001950095FFF7CDFFFF236580637225706F
:1083B00037BD000010B50C4904004A88002A09D0D6
:1083C0008B89002B05D00020CB8A0222834201D06A
:1083D00010BD012213000A20434300204032C8543C
:1083E000C81842800472F3E7CA64FF1F0023438069
:1083F00003707047094B00211A0010B55C88002CEF
:1084000006D01C79844203D10A234B43D01810BDF7
:1084100001310A330329F1D10020F8E7CA64FF1FB4
:1084200010B50400407A03F073FAFF23637210BDA5
:108430007047043010B580B203F072FB002803D0FF
:108440000421494203F0E4FB10BD000070B5002593
:10845000104CA0682580A581A580A84202D003F019
:10846000F7F9A56000250C4C0C4B606D1D802300B6
:1084700058331D70A84202D003F0EAF96565002563
:108480006068002801D003F0E3F9013508340A2DB3
:10849000F6D170BD9065FF1F3465FF1F8465FF1F17
:1084A00070B5041E09D1054D2880A881A880A86850
:1084B000002802D003F0CCF9AC6070BD9065FF1FBE
:1084C000F0B54B8885B00193002343600A7905001D
:1084D0000F00022A00D07BE0CA88032A17D98B68D4
:1084E0005E7819783602DC78D8790E4399781B7A51
:1084F00024021B020C43034353495BBA0B80331D18
:1085000093421ED1042C04D0631F022B0ED90120EC
:1085100015E0019A4D4B1201D35A002B06D0019859
:10852000FFF7BEFF4A4A1369013313610421B8689B
:108530002E812C80494203F06BFB6860002005B05F
:10854000F0BD434D042C06D0631F022B0FD9EB68FE
:108550000133EB60DBE7019A3C4B1201D35A002B4D
:1085600005D00198FFF79CFF2B6901332B61374B36
:1085700030000293019B029A1B0101930023019991
:108580008C468B52130063449C8003939E81FFF7BB
:1085900050FF039B041E986016D00421B86849421E
:1085A00003F036FBFA880100043A200003F0F8F8E3
:1085B0000199029AFB888A5A043B9B18029A8B52B3
:1085C0002B6801332B60A2E7AB690133AB619EE7F7
:1085D0001E4B0293019B1E01029BF35A002B2DD0D0
:1085E00002998C19A068002828D0012A26D1FA887F
:1085F0009B189BB27352A189994217D39B1AC0183A
:10860000B96803F0CDF8029BA289F35A934200D0D7
:108610007DE700222B81A3882B80A3686B60029BDF
:10862000F2520B4A53680133536070E7084A93686B
:10863000013393600198FFF733FF68E7044A5369F9
:1086400001335361F6E7C046FA64FF1F9065FF1FD0
:108650000065FF1F70B5051E15D10B4C0B4B188024
:10866000230058331870606D002802D003F0F0F832
:108670006565250050356068002801D003F0E8F8F2
:108680000834AC42F7D170BD3465FF1F8465FF1F0D
:10869000F0B51700A12285B0920001934243394BF7
:1086A00006001B680C009B18D933FF331D78FDF7BB
:1086B00041FF0430854204DD3000FDF73BFF04300C
:1086C000C5B2BD4207D33A0000213000019B03F040
:1086D0006FF805B0F0BD2900380003F0F9F9230068
:1086E000C6B250331E700393019B290063653800A6
:1086F00003F09EF8CBB20293002B02D0039B01360D
:108700001E7000262300503303931B78B34204D815
:10871000606D002831D10020DBE7029A2800002A92
:1087200004D0013B1000B34200D02800F700E71945
:10873000387003F005F9786000280ED03A78019976
:1087400003F02EF8019A3B780136D3180E4A0193B4
:10875000D369F6B20133D361D4E7039B1870606527
:10876000A74205D1084A1320D36A0133D362B0E788
:10877000606803F06DF80834F2E703F069F800234D
:108780006365C8E73409FF1F0065FF1FF7B50D00DB
:1087900007000421686803F03BFA2B89040003708A
:1087A0002B891B0A43702B8883702B881B0AC3708C
:1087B0002E8902250436F6B2F42E15D81B4B9F42A3
:1087C00014D10C2003F0ACF81135011E0CD090230D
:1087D00003708E3B0371043B4380154B8460C6805D
:1087E000187803F05DF900252800FEBD5C237B436B
:1087F000104AD3180093583301931B78002B0FD1E4
:108800000300320038000099FFF742FF019B05008A
:108810001B78002BE8D13800009903F011F9E3E749
:10882000054A0725536A01335362DDE7FEFF000066
:10883000F864FF1F3465FF1F0065FF1FF0B587B0A8
:10884000009017200F0016000193FFF7F2FD13258B
:10885000041E19D00C98031E02D00199201D9847C0
:10886000030AE370052302AAA070043090812770E8
:108870000098667003A993800494FFF787FF051E94
:1088800002D0200002F0E4FF280007B0F0BD000095
:10889000F0B587B01F000CAB1B7803910593012145
:1088A0000DAB06001C78049200F0D6F814250028C1
:1088B00021D02000FFF77EFD0135041E1BD0114999
:1088C000059B0A7803700132D2B2131EC68001D113
:1088D00001231A000B7022713000049B039900974A
:1088E000FFF7ACFF051E09D1230021000648074A07
:1088F000093302F0D5FE280007B0F0BD00236380E5
:108900002370F8E7FC64FF1F8B83001130750000B3
:10891000F8B505000E00064C064F2368002B02D068
:108920003100280098470434BC42F6D1F8BDC04657
:10893000A065FF1FB465FF1F0123064A5B425380F9
:10894000002313715362044A136053609360D36031
:1089500013617047B465FF1FA065FF1F020000236D
:1089600010B506499C000859002801D1625010BD7D
:108970000133052BF6D11320F9E7C046A065FF1F90
:10898000034A5388181A43425841404210407047E6
:10899000B465FF1FF0B585B002930AAB1F780CAB2E
:1089A0001B88009008000E0001920393FFF7E8FF78
:1089B00005001120002D1BD10E48FFF7E1FF040038
:1089C0001520002C14D006220B99A771E01D02F08F
:1089D000E7FE019B30002371029B29006371009B1D
:1089E00066802370039B6562E381FFF791FF280097
:1089F00005B0F0BDFFFF000010B5FFF7C1FF040098
:108A00000220002C12D060880121FFF781FF606AEC
:108A1000002801D003F0F4F828220021200002F001
:108A20001FFE012300205B426380207110BD000007
:108A300030B5074A074C5588010013780020A5423D
:108A400004D05B1A59424B415842104030BDC046D9
:108A5000B465FF1FFFFF0000084A10B501230C009A
:108A6000904208D0FFF78CFF031E04D00379234007
:108A70005A1E9341DBB2180010BDC046FEFF000035
:108A8000024B1879431E9841C0B27047B465FF1F6E
:108A900070B504000D001600FFF772FF002804D126
:108AA0000D4B9C4200D0143070BD416A0379052003
:108AB000002907D012221A40102A02D10520002EC8
:108AC000F2D10F20DB06EFD5897E0C20A942894127
:108AD000494249420840E7E7FEFF0000030010B5A5
:108AE000002800D110BD0348034A41889142F9D0C3
:108AF0009847F7E7B465FF1FFFFF0000002330B57C
:108B0000C45CCD5C6C40D4540133102BF8D130BD23
:108B10000F23002210B5C45C64002243CA54C25C17
:108B2000D209013BF7D210BD0200010010B520327E
:108B3000103102F0DDFE10BDF0B58BB003901020B7
:108B400005931700049102F08BFE0090102002F0B4
:108B500087FE009B13240190002B05D000280CD128
:108B60001324009803F04CF8019B002B02D018004E
:108B700003F046F820000BB0F0BD102002F070FEAC
:108B80000600102002F06CFE13240500002E00D118
:108B9000AEE0002819D01022002102F061FD320061
:108BA0002900039802F0A4FE041E0ED133787F2B17
:108BB00051D830000099FFF7ABFF009B1B787F2B4B
:108BC00053D801990098FFF7A3FF300003F018F87D
:108BD000002D02D0280003F013F8002CC1D1102082
:108BE00002F03EFE0600102002F03AFE0290002E37
:108BF0007CD0002878D03A000F32230001251211D2
:108C000005D00F333B4015B25A4253411BB26A1E86
:108C10001201002B33D0049BD2B298180099029A0B
:108C2000FFF76CFF013D10220021300002F018FD1B
:108C3000ADB2049F2D017D19AF4242D0002C33D03C
:108C4000300002F0DDFF029B002B00D189E7180005
:108C500002F0D6FF85E729003000FFF759FF280012
:108C60002549009AFFF74AFFA7E729000098FFF778
:108C70004FFF28002049019AFFF740FFA5E70F2189
:108C80000F4004998A18D9B28F4208D9D15C06A83E
:108C900019540133102BF6D1029A0199C0E7791AC1
:108CA00048424141C901F2E73900300006AAFFF706
:108CB00025FF3200039806A902F01AFE10370400BF
:108CC000BAE7002CBCD13000029906AAFFF716FFC4
:108CD000320006A9039802F00BFE082204003100BE
:108CE000059802F05DFDABE71324A9E71324AAE77A
:108CF000002800D06EE733E7B0BE0011F0B58BB0AE
:108D00000F0016000225009000283FD0002A3DD019
:108D10000B1DDBB21800029302F0A2FD1135041EF8
:108D200034D0FDF747FD05003A000099201D02F000
:108D30009FFEEBB20393E3702B0CDBB22F0A009380
:108D40006370FFB22B0E2370A7700193FDF72CFD0B
:108D50001022010006A802F08BFE2100029A04AB4B
:108D600006A8FFF7E9FE051E0DD1039B082233700C
:108D7000009B04A9B370019B7770F370301D02F063
:108D800077FEFDF71DFD200002F03AFF28000BB032
:108D9000F0BDF0B58FB00D00149E039004920593C2
:108DA000002A03D1022420000FB0F0BD002EF9D01C
:108DB0000398FFF7E5FD1424071EF4D0727833788A
:108DC00012021A43B3781B041343F27812061A43B3
:108DD000036A0192934201D30133E3D1002D03D002
:108DE0003B7901249B07DED50822002106A802F06A
:108DF00037FC059B13240433DBB21800029302F006
:108E00002FFD051ECFD0059A0499043002F030FEE4
:108E100004223100280002F02BFE3900102210310C
:108E20000AA802F025FE2900029A06AB0AA8FFF75D
:108E300083FE041E0FD1082206A908A802F018FE1E
:108E40000822311D08A802F003FE012807D101996C
:108E50000398FDF7C9FC280002F0D2FEA3E7012425
:108E6000F9E7000070B51C4C05002368181E10D0EF
:108E7000002D14D11A78002A0CD1981C083202F067
:108E80008FFC02F08DFD0135002808D123681D708C
:108E9000012070BD0A331800082202F081FC23680B
:108EA000002BF5D0122002F03BFD061E0DD0C12391
:108EB00021680370457002311022023002F070FC0C
:108EC00023683100587802F0EBFD206802F098FE2C
:108ED00000232360DCE7C046DC65FF1FF8B5040013
:108EE0002020FDF755FB0D4EA700BB590500002BB8
:108EF0000DD000280BD0D878FF2809D108492A00C6
:108F00000C55F35907480333611802F0C9FBF8BD4B
:108F1000290002F0CDFB0028F0D1F8E7F865FF1F2B
:108F2000E065FF1F35A1001170B5064D840063593F
:108F3000002B05D0D87802F0EBFCFF226359DA70E1
:108F400070BDC046F865FF1F70B506008CB00C0000
:108F5000150000213022684602F082FB3100102209
:108F6000684602F085FD1D2021000322684402F0BE
:108F70007FFD6846FFF7D8FD2D210400032228005D
:108F8000694402F075FD20000CB070BDF0B507001B
:108F9000160097B001931CAB1D7830221EAB0091D8
:108FA0000AA800211C7802F05BFB102239000AA8F5
:108FB00002F05EFD1022002102A802F051FB072200
:108FC000310002A802F054FD072202AB9818631E7C
:108FD0009C41019902F04CFD02AB9C732B005A1E80
:108FE000934102AAD3730021102206A802F038FB95
:108FF00006221D9907A802F03BFD1A2002ABC018FB
:1090000006221F9902F034FD102200990EA802F0EA
:109010002FFD102202AB0EA908781C78013A60409F
:10902000D2B2087001330131002AF5D10AA8FFF746
:109030007BFD102212A904000EA802F0B1FB102241
:1090400006AB0EA908781D78013A6840D2B20870C4
:1090500001330131002AF5D10AA8FFF765FD044369
:1090600010222098E4B212A902F002FD200017B0ED
:10907000F0BD70B50E0014008CB0010010226846DF
:109080001D0002F0F5FC3100082204A802F0F0FCFB
:109090002100082206A802F0EBFC6846FFF744FD19
:1090A00004001022280008A902F0E2FC20000CB005
:1090B00070BDF8B506000D0000243719AC4200D38E
:1090C000F8BD02F015FB030A3B70631CDBB20137ED
:1090D0009D4203D90234F054E4B2EEE71C00EDE700
:1090E00073B506000C000225002819D0002917D0FE
:1090F000032101A8FFF7DDFF6B469A793F231A4051
:10910000013313436A463000937101A92200FFF72F
:109110001BFF051E04D10322E01C01A902F040FB45
:10912000280076BD03785807DA08C00FD200800007
:109130009B0710439B0F1843C0B2704707230B4097
:10914000C908C9000B4303707047000070B50400E4
:10915000FFF7EAFE134DA4006359002B21D0186AD3
:10916000002801D002F04CFD2B59986E002801D048
:1091700002F046FD2B59D86E002801D002F040FDC8
:109180002B59186F002801D002F03AFD2B59586F67
:10919000002801D002F034FD285902F031FD0023EF
:1091A0002B5170BDF865FF1F0E4B8000C35870B582
:1091B0000C00002B0FD09D68002D0CD02B78201DAB
:1091C0000B706B784B70A97CFFF7B8FF2B7E237276
:1091D0006B69E36070BD10220021200002F040FAAC
:1091E000F8E7C046F865FF1F014B18607047C0469E
:1091F000F465FF1F074A03008000825810B5002A5B
:1092000006D0D088984203D1012901D1FFF79EFFF3
:1092100010BDC046F865FF1FF0B5264E95B087001B
:109220000B93BB590500099112200A92002B31D0F3
:10923000D888FFF7A5FB04001420002C2AD02800B2
:1092400010A9FFF7B1FFBB591E781D6A002E23D06D
:109250000895FDF7EFFA07000020FDF7F1FA0790F7
:10926000A379E61D069310AD0CA9089800F0E2FA68
:109270000EA9280000F0D7FA0B9B0A990493069BCD
:1092800009980293079B0396019300970EAB0CAAD3
:10929000FFF77CFE15B0F0BDFDF7CCFA069030006C
:1092A000FDF7CEFAE31DA779079310AB06000893EC
:1092B000DAE7C046F865FF1F30B50C4C85002A5927
:1092C000030085B00120002A0ED018006946FFF780
:1092D0006BFF2B591A78D888054B002A00D1054B13
:1092E0006A46072100F0D9FB05B030BDF865FF1FC5
:1092F000279800113598001130B5094C850029597F
:1093000085B010226846253102F04AFA2A59112107
:10931000044BD0886A4600F0C0FB05B030BDC046A3
:10932000F865FF1FD198001130B5094C8500295907
:1093300085B010226846353102F032FA2A591121DF
:10934000044BD0886A4600F0A8FB05B030BDC0468B
:10935000F865FF1F0F990011F7B54D4F86001020DB
:10936000F4590D0002F07CFAF3592062186A1322B6
:1093700000286CD0033A29009C6802F011FAF359D6
:109380001A780192002A58D11E6A227D317B9446B8
:1093900051400122019F114201D167461740217DB2
:1093A000914339432175377B4F40BC4660460027C7
:1093B000800701D44F081740012102208F40227DF1
:1093C00082433A432275377B5740BC4660460027AC
:1093D000400701D497080F400420227DBF0082433C
:1093E0003A432275627D002794466046727B424074
:1093F0000A4201D167460F400121627D8A433A4308
:109400006275777B5740BC4660460027800701D4D1
:1094100057080F400220627D7F0082431743677523
:10942000767B00227E40760701D4BA080A400426E3
:10943000617D9200B1430A4362756A78002A08D0C0
:109440006278002A05D005220533DA770022100061
:10945000FEBD04222979114205D1A17C114202D11D
:109460000533033AF1E7019A21782C78002A02D1DA
:109470000A002100140018220429E8D8042CE6D898
:1094800005206043034A05331218525CDDE7C046ED
:10949000F865FF1FC0BE001110B50A001121024B74
:1094A00000F0FBFA10BDC0466B9900110B0030B5FF
:1094B00087B001AD2B806B4604001100981D082277
:1094C00002F06EF92A000B212000024B00F0E5FAB1
:1094D00007B030BD9399001110B50A001121024B5D
:1094E00000F0DBFA10BDC046E799001113B50B0080
:1094F00011006A4613706B4604000622581C02F0E5
:109500004FF96A4608212000014B00F0C6FA13BD4E
:10951000079A001110B50A001121024B00F0BDFAA4
:1095200010BDC046579A00117FB505000B4BAA002D
:10953000D4580800002C0FD0666F237FE288217872
:109540000396266F0296E66E0196A46E0094FDF7D0
:1095500009FC2800FFF7FAFD7FBDC046F865FF1F34
:1095600010B51721FFF7E0FF10BD000070B50A002D
:109570000D00064B0221040000F08FFA0600297846
:109580002000FFF7D1FF300070BDC04637990011B1
:1095900070B586B000236A461370836804001D7896
:1095A000681E0A2859D801A902F0EAFA06063337DC
:1095B0003B3F43474B4F5300180000F042F906234E
:1095C00012284BD000281BD16088FFF7D9F9082357
:1095D000002813D04279002A47D1264B1A78072356
:1095E00012070BD5244B1A680723002A06D01668E9
:1095F000002E03D0290001AAB04703006A46137069
:109600006B461B786088002B2AD1FFF767FC06B0F9
:1096100070BD180000F06CF9D4E7180000F087F96D
:10962000D0E7180000F093F9CCE7180000F0ADF98E
:10963000C8E7180000F0C3F9C4E7180000F0F6F915
:10964000C0E7180000F0F6F9BCE7180000F013FAC4
:10965000B8E7180000F013FAB4E707236A4613705E
:1096600069466088FFF782FFD1E70523012AC5D14B
:10967000024BB8E78564FF1FF065FF1FF465FF1F0D
:10968000F8B52C4F8600F35904000D00002B40D094
:10969000DA8882423DD15A78062A33D11A78002AD4
:1096A0002ED0012099681A6A097D014206D0157BE7
:1096B000054203D007225A700120F8BD0220014262
:1096C00004D0157B054201D00922F4E704200142B1
:1096D00004D0127B024201D00B22ECE7164B1B6830
:1096E000002BE9D05B68002BE6D020009847BB59DF
:1096F00000215B78122BDFD12000FFF715FFDBE79D
:109700000E4BECE7112A04D1002900D032252900A4
:10971000F2E7002D08D12000FFF732F9002803D02E
:10972000102302791343037121002800FDF798FAF2
:10973000C2E7C046F865FF1FF065FF1FF465FF1F15
:1097400070B50E4E8500AB590400002B13D01B786A
:10975000002B11D10A4B1B68002B04D05B68002B37
:1097600001D02000984773595B78122B03D1002158
:109770002000FFF7D9FE70BD024BECE7F865FF1F34
:10978000F465FF1FF065FF1F094B8000C3581020D0
:10979000002B0CD01A6A002A09D09B68002B06D037
:1097A000127A1B7E101C9A4200D9181CC0B2704756
:1097B000F865FF1F70B503000D0014000220002A99
:1097C00030D000292ED013700B78081D53704B78C1
:1097D0009370FFF7A7FCE070012002212B7A237120
:1097E0006B7B034063716A7B0A40134304226371FD
:1097F0006E7B1640334363716E7BF608F60033438D
:1098000063712B7B0340A371287B014000200B4335
:10981000A371297B0A401343A3712A7BD208D2008B
:109820001343A37170BD10B50A0001000120FFF7BA
:10983000C1FF10BD10B50A0001000220FFF7BAFFFA
:1098400010BD70B506000C000220002E30D000299B
:109850002ED07378201D0B70B3784B70F178FFF722
:109860006DFC01223579257271794B100800134087
:10987000934010400343881010408000C908034300
:10988000C9000B436373B1794B1008001340934038
:1098900010400343881002409200C9081343C900D6
:1098A0000B4321202373FCF773FE854201D2122063
:1098B00070BD2220257AFCF76BFE8542F7D823780D
:1098C0001820042BF4D86378012BF1D80020EFE79F
:1098D000030010B50220002909D0002B07D0032275
:1098E000481C0A7019000D3201F05AFF002010BD0B
:1098F00003000222080010B5002B06D0002904D076
:109900000E32591C01F04CFF0022100010BD030064
:1099100010B50220002909D0002B07D00422481CD2
:109920000A7019000C3201F03BFF002010BD10B589
:10993000FFF7DEFF10BD03000220002906D0002B38
:1099400004D0052200200A701B784B70704703007A
:109950000220002B08D0002906D05B7800200B7075
:10996000013B082B00D918307047030010B50220C6
:10997000002909D0002B07D00622481C0A701900C4
:109980000A3201F00DFF002010BD10B5FFF7B0FF47
:1099900010BD02000B00022010B500290ED0002AD5
:1099A0000CD007211970118859701188090A997013
:1099B00011180822D81C01F0F3FE002010BD03008E
:1099C0000A00022010B5002B0CD000290AD099788B
:1099D0005878090201431180901CD91C082201F01B
:1099E000DFFE002010BD030010B50220002909D0C1
:1099F000002B07D00822481C0A701900921801F0A9
:109A0000CFFE002010BD02000B00022010B500297F
:109A10000BD0002A09D00921197011781818597033
:109A2000511C062201F0BCFE002010BD10B5FFF74E
:109A30005FFF10BD02000B00022010B5002A09D004
:109A4000002907D05178197011180622581C01F00E
:109A5000A7FE002010BD030010B50220002909D088
:109A6000002B07D00A22481C0A701900063201F0A8
:109A700097FE002010BD10B5FFF73AFF10BD0200A1
:109A80000B00022010B5002A06D0002904D01800CF
:109A90005178FFF753FB002010BDF0B585B01700DB
:109AA0001E006A4606230500080091819380FEF798
:109AB000C0FC1324011E02900CD03800B047041ED5
:109AC00005D1280001A9FEF76FFA041E02D0029802
:109AD00001F0BEFE2800FFF701FA200005B0F0BD3E
:109AE000F0B504008BB0019115000021102202A8EE
:109AF00001F0B6FD334EA700B85900283CD0C3880A
:109B0000A34239D10378002B36D14278062A18D1E6
:109B100002000100553235310C3006ABFFF7A9FACF
:109B2000002829D12000FFF72FFE020006A902A875
:109B300001F036FE200002A901F06AFE01200BB000
:109B4000F0BD816E002917D00B8A112A28D19D42C1
:109B50000ED101981231093A01F07AFF012807D19C
:109B6000BB5920009D6EFFF70FFE29000200DEE7C3
:109B700032212000FFF7D8FC2000FEF701FF061E6F
:109B80001BD0416A002918D00B8AAB4215D108229C
:109B90000198123101F05CFF01280ED1716A0AE0D0
:109BA0009D42E9D108220198123101F051FF0128AC
:109BB000E2D1BB59996E8A7EB9E7200001F028FFF7
:109BC000BCE7C046F865FF1FF0B56B4D87007E59B6
:109BD00085B0337802900393002B00D087E0B36800
:109BE000346A01937078062817D101221B7D134235
:109BF00002D0217B114218D10222134202D0217BD4
:109C0000114251D10422134203D0237B134200D0CE
:109C10008BE0019B5A7DEB5991E007380428F8D876
:109C200001F0AEFF032E42678300B36E002B03D119
:109C30001C2001F015FEB066EB599C6E002C1CD068
:109C400010220021200001F00BFD0298FFF79CFD7F
:109C500001002000FFF72DFA01F04AFD20822000CC
:109C600008211230FFF725FA0298FFF78DFDA07644
:109C7000EB592100D888FFF70FFC0822EB591CE0B4
:109C8000B36E002B05D01A00198AF0881232FFF744
:109C90000DFC0222019B197DEB5911423DD0207B26
:109CA00010423AD0073208E0F488FCF7DBFD0100EF
:109CB0002000FFF711FC0A22EB595A70029B9C000E
:109CC0002A595378073B042B11D8D088FEF758FE49
:109CD00000284ED0C3895A08D2182849029B0298FE
:109CE000CB542B5941180433254801F0D9FC05B059
:109CF000F0BDFCF79FFD03000120834201D100204D
:109D00000393EB59DE88FCF79BFD039902003000BA
:109D1000FFF7ECFB019AEB59117D042211420CD0A4
:109D2000217B114209D00B22C7E7F688FCF73CFDE6
:109D300001003000FFF7EEFB6BE7019A527D012135
:109D40000A4204D0607B084201D00C22B5E7022110
:109D50000A4204D0607B084201D00E22ADE7042104
:109D60000A4204D0627B0A4201D01022A5E71222E7
:109D7000A3E7FA225200B0E7F865FF1FFC65FF1F5A
:109D80003FA1001110B5064B1A78042310001840AB
:109D90001A4200D00348FFF727FA002010BDC04642
:109DA0008564FF1F4843FF1F70B50400FFF7D4FA16
:109DB000051E43D12000FFF77FFA234EA400A059CF
:109DC0008268937CDB0708D50321036A1B790B406B
:109DD000012B02D1017F0B430377431DD97F8B1EDB
:109DE000022B0DD8022900D00121C088FCF790FF7A
:109DF000042133591A7F59700A431A77280070BD1D
:109E000001290CD102231022437000210C3001F0F3
:109E100027FC305910213530FFF74BF9EEE70529C3
:109E2000ECD10223D118437010220C3001F0B8FCA1
:109E300004233259117F0B431377EAE708251828CA
:109E4000DCD1053DDAE7C046F865FF1FF0B58BB001
:109E5000059143887E4F9E00F45915000493002C11
:109E600015D1012902D000200BB0F0BD101D57788C
:109E70001678FFF757F9EB68320002932B7A0499B2
:109E8000019300903B002000FCF70CFFEBE7E38818
:109E9000049A934201D00820E6E72378012B00D1F1
:109EA000D4E0059B581E092800D9CFE001F068FED8
:109EB00005CE0A29CC506C859AB229000498FFF788
:109EC00073FFD1E7200029001022453001F068FC23
:109ED000B9594B78042B02D1013B4B70C3E70B00FF
:109EE0000A00253335320C310498FFF795F90498B0
:109EF000FFF702FA0522431E9841BB59C0005A7071
:109F0000B2E7200029001022553001F049FC049BE3
:109F10004F4C9D00295904980A0006AB55320C316C
:109F2000FFF77AF929591022453106A801F090FD72
:109F3000012808D10498FFF7F7F90590002804D10B
:109F400006222B595A7005988EE708230593FAE7E5
:109F500063780C2B7AD1E36E002B03D11C2001F027
:109F60007FFCE066BB59D86E00286FD01022290014
:109F700001F016FCBB590498DC6EFFF705FC0D22BE
:109F8000A076BB595A706EE7E06E00285ED0637809
:109F90000D2B5BD12B8808220382A91C123001F003
:109FA000FFFBBB599A68517D0222114226D0186AE4
:109FB000407B104222D00C32E4E763780E2B45D16F
:109FC000236F002B03D1162001F04AFC2067BB59F8
:109FD000186F002803D01022290001F0E1FB0F22A6
:109FE000BB59CFE763780F2B30D1206F0622691C55
:109FF000103001F0D5FBBB599A68517D0422114203
:10A0000003D0196A497B1142D5D100210498FFF78A
:10A010008BFA28E7636F002B0DD0BB59586F0028CF
:10A02000F3D01022290001F0BBFB0122BB595242A0
:10A030005B6F1A61E9E7142001F012FCBB596067FD
:10A040005B6F002BE9D126E72978DFE707200BE7D4
:10A05000F865FF1F10B5064C207001F091FB06213A
:10A060002078FDF791FF0348FEF778FC10BDC0464D
:10A070000B66FF1FF591001100200BB270B50D00AB
:10A08000834216DA264B187801F0BAFB041E0DD075
:10A090000378922B0ED0A02B37D0224B1878FF28B4
:10A0A0003AD0210001F0FCFC002835D180200002CC
:10A0B000684070BD43780E2B0BD03E2BEDD18378DA
:10A0C000052B12D0082BE8D181798088FFF7D8FAC8
:10A0D00008E0154B82889A42DFD183681878591CB2
:10A0E000FEF7C0FE002817D1D7E7104B1B785B079F
:10A0F00012D50F4B1B68002B0ED09B68002B0BD08A
:10A10000C289811D80889847ECE7FFF741FAA06873
:10A11000002801D001F09CFB200001F099FDC5E76B
:10A120000B66FF1F4143FF1F182000008564FF1FBF
:10A13000F465FF1F10B50078FFF712FA10BD10B5D7
:10A140000078FFF7FDFA10BD0C234343084A10B511
:10A150009B185A68002A03D0012901D1904710BDED
:10A160009B68002BFBD00029F9D19847F7E7C04640
:10A170002866FF1F01238340094A10B5946B1C43D6
:10A180009463506B98435063D46B2000984301292B
:10A1900001D120001843D063116B0B43136310BD32
:10A1A00000800040F0B500240127154B85B0DA6B24
:10A1B000144E03921A6C0192DA64019BE3403B4215
:10A1C00017D0039DE5403D400295E5B20299280075
:10A1D000FFF7BAFF316A736A002908D03900002BF3
:10A1E00001D0029979402800FFF7C4FF01E0002B5D
:10A1F000F9D101340C36172CDFD105B0F0BDC046C3
:10A20000008000400C66FF1F064B01215A68C240C7
:10A210000A4204D01B68C3401800084070471B6DF9
:10A22000F9E7C046008000400122064B8240002929
:10A2300003D0D9680A43DA607047D9689143D9607E
:10A24000FAE7C0460038004030B5032444430F4BC2
:10A25000E25C1B199C785D7801232D1B0135AB4016
:10A26000013BA340A140DB430C00122807D808495A
:10A2700092005218116819402143116030BD054AFF
:10A2800011680B4023431360F8E7C04607BF001175
:10A2900008F0004014F00040C21F70B5D4B206238D
:10A2A000092C0BD80125084C9540002908D0002125
:10A2B000FFF7CAFF23682B4323600023180070BDFB
:10A2C0002368AB43F8E7C04600380040214BF0B5A7
:10A2D0001B185B78022B21D1032444431E4A1F4ED6
:10A2E000A35C12199478012215008540B76B013CDC
:10A2F000E4B23D43A240B563194C122815D89B0027
:10A3000000290CD117495B1899680A439A60012308
:10A31000205C154A834011680B431360F0BD11495E
:10A320005B18996891439960F1E70E4B00290DD1B4
:10A3300059690A435A61225C1328E8D00123203A64
:10A3400093400A49086803430B60E7E75969914362
:10A350005961F0E70C66FF1F07BF00110080004045
:10A360004CBF001100F00040A0F00040A4F00040FD
:10A37000F8B500241B4E1C4D1C4B1B5D012B1FD13F
:10A38000194A9269E2401A420BD00122B256934018
:10A390002200143AD2B2022A09D815494A69134355
:10A3A0004B61013402360C35172CE5D1F8BD002283
:10A3B000B2560F499200521891680B439360F0E730
:10A3C000022BEED1E7B23800FFF71EFF0123584001
:10A3D000C1B23800FFF77AFF3800FFF715FF687742
:10A3E000DFE7C046D9BE00110C66FF1F0D66FF1FD8
:10A3F00000F00040012202388240054B002903D0C2
:10A4000059690A435A617047596991435961FAE79A
:10A4100000380040F8B50E0001210F008740114AB6
:10A420000400D368FD43BB43D360831E8B4201D835
:10A43000FFF7E0FF00212000FFF72EFF0A4A0B4B39
:10A440005168012E05D139431B1951605E700020FF
:10A45000F8BD2940516002221C1962709A691540AA
:10A460009D61F4E700380040008000400C66FF1F4B
:10A47000012210B58240074B002906D019680A4313
:10A480001A600121FFF7C6FF10BD196891431960DA
:10A49000F7E7C046008000400C2370B50025434319
:10A4A0000A4A29009B181D70094B04001B185D7097
:10A4B000FFF7B0FF0123A340064928000A681A43AA
:10A4C0000A6005490A689A430A6070BD2866FF1F42
:10A4D0000C66FF1F348000403080004070B50400DF
:10A4E0000E00FF2813D003250540FFF7D5FF084ACB
:10A4F000A3089B009B183F22ED00AA40AE401968BC
:10A5000020009143314319600121FFF78DFE70BD9A
:10A5100018380040F8B50C244443134B0500E418E8
:10A520006368002B03D1A3681220002B1AD00222EB
:10A5300001270E4B00215B195A7028002770FFF786
:10A5400069FF63681E1E08D0A3683E00002B04D07C
:10A550002800FFF759FE4640F6B228003100FFF709
:10A5600009FE0020F8BDC0462866FF1F0C66FF1FCD
:10A57000F7B5C420FF222B4B8000195800249143CB
:10A580003F3A0A431A508022274F5202274E1A6040
:10A59000274B1D5D002D21D0A31E012B03D80121C7
:10A5A000E0B2FFF727FF012D18D11F4B9B69E34055
:10A5B0002B4213D0E3B218000193FFF725FE0100F0
:10A5C0000198FFF755FFE3B2143B022B1DD8012180
:10A5D0007156184A8D405369AB4353613B7F002B42
:10A5E0000DD0E5B22800FFF795FF2800FFF70CFE1D
:10A5F0007B7F0100834202D02800FFF7A5FD0134D4
:10A600000C370236172CC3D1F7BD01210023715638
:10A61000F3568D40074A9B009B189A68AA439A609C
:10A62000DCE7C04600E100E00C66FF1FD9BE001168
:10A630000D66FF1F00F0004010B501210400FFF778
:10A64000E9FE0123044A002011194B70A3409169CF
:10A650000B43936110BDC0460C66FF1F70B50E0022
:10A6600015000400FFF718FF0C236343094A20007C
:10A670009B189D605E60FFF74DFFF021064B074A77
:10A680008900051E5A5002D02000FFF705FF280060
:10A6900070BDC0462866FF1F0000FF1FA5A1001166
:10A6A00070B5134D07202C78002C1FD19822210063
:10A6B0005200280001F05CF90123C420FF222B7016
:10A6C0000C4B80001C635C630B4B1C605C600B4B91
:10A6D000195891433F3A0A431A50802252021A6095
:10A6E0000D20074A074901F04BF9200070BDC04614
:10A6F0000C66FF1F00800040A0F0004000E100E079
:10A7000071A5001171A30011030010B50620072BDD
:10A7100009D8054A137001F03BFAD7210020034BFA
:10A72000034A89005A5010BD7043FF1F0000FF1FED
:10A73000D91AFF1F70B51D0002240C2910D8094A30
:10A74000CA40D2070CD5FBF72FFF041E08D1059A8B
:10A7500004992800FBF744FFFCF7B2FDFFF712FB5A
:10A76000200070BD1210000030B50D7802232C00BF
:10A770009C43184201D02B431C0008252300AB4307
:10A78000284201D02B00234320241D00A543204252
:10A7900001D01C4325002A230D70184204D01178E3
:10A7A0001E3B0B43137030BD0028FCD10C211378E5
:10A7B0008B43F7E7F8B51D0006AB1B88140007AA0A
:10A7C0000E000B201778002B27D10A78022A49D1D6
:10A7D0004A68507811780002244A084380180428F7
:10A7E00040D801F0CDF903121D1B2300F06801F0E1
:10A7F000E7F9021CC0B2B84200D93A1CD2B220001C
:10A80000F1682A8000F0CCFF06E00222F3681B8882
:10A810002A8023701B0A63700020F8BD0622EEE731
:10A8200001232B80F3681B782370F5E7F368002B76
:10A8300016D008222A801A8822701A88120A62709A
:10A840005A88A2705A88120AE2709A8822719A88ED
:10A85000120A6271DA88A271DB881B0AE371DBE7F6
:10A860002B80D9E701202B80D7E7C04600D6FFFF19
:10A87000F7B516000A781D0008AB1F880C000123ED
:10A88000022A18D14A685078117800022B4A0843EE
:10A89000801803280FD801F073F902254439E068C5
:10A8A00001F08EF9C0B20723B84204D37B1901939B
:10A8B000152B02DD0D231800FEBDE0682A003100D3
:10A8C000C01900F06DFF6B4600209B88E268D054F1
:10A8D0001B4B1B68834203D01B68834200D0984700
:10A8E0000023E8E70B23002FE5D1022DE2D1737896
:10A8F00032781B021343E2681380114B1B68002B54
:10A90000EED01B68002BEBD00120E8E70B23002FD3
:10A91000D1D1062DCED12A003100E06800F040FFF1
:10A92000DEE70B23002FC6D1012DC3D1327875335A
:10A93000012AC0D8E3681A70D2E7C04600D6FFFFEC
:10A940001868FF1F70B50C001500072837D801F0F4
:10A9500017F9041436361B36242E182015290BD867
:10A96000184E16220021300000F07AFE2200290045
:10A97000300000F015FF002070BD18200229FBD127
:10A980001288114B1A80F6E718200829F4D10A0022
:10A990000E48290001F0B4F8EDE718200129EBD1A9
:10A9A0000B4B10780B49DA69FFF7DEFEE3E718205E
:10A9B0000129E1D1064B10780749DA6BF4E7022050
:10A9C000DAE7C0460068FF1FEE43FF1FE443FF1FA6
:10A9D0007443FF1F9C43FF1FBC43FF1F030010B5C0
:10A9E0000020DB0704D50721024A034800F08CF859
:10A9F00010BDC04664BF00117443FF1F054A030029
:10AA00001068002803D082889A4201D1806870477C
:10AA10000068F6E7106AFF1F0A88030008009A42E0
:10AA200004D08A8804309A4200D000207047000089
:10AA3000F8B5F22200230D4F0D4E79680500424310
:10AA40003370994200D07B600A4C0021200000F056
:10AA500007FE00231A007C60AB4202D10020337055
:10AA6000F8BD01332280DBB2F234F5E7086BFF1F3B
:10AA7000066BFF1F146AFF1F73B56B46019006003B
:10AA8000684615001980FCF74DFF041E11D1002DFA
:10AA90000FD07689002E11D00C2000F0E1FE0028A6
:10AAA0000ED0084A0460136886808560002B02D1AE
:10AAB0001060200076BD1A001B68F7E70224F8E753
:10AAC0001324F6E7106AFF1F012100220A4B10B57C
:10AAD00049420A4C198099809A719A70084B2070EB
:10AAE000012019805A60FFF7A3FF2078FCF778FF58
:10AAF0000448FDF733FF10BD2068FF1F106BFF1FD8
:10AB0000086BFF1FB5AB0011022310B5002802D05F
:10AB1000FFF7B2FF0300180010BD0000030010B5DE
:10AB20000020DB0704D50421024A0348FFF7A4FFF5
:10AB300010BDC04678BF0011F443FF1FF0B50E26CC
:10AB400087B003930CAB1F8802ABF6180500080012
:10AB500031000292FDF768F804000120002C0FD0AC
:10AB60003088FFF74BFF03000E20002B08D05E68F3
:10AB7000002E05D021002800039B029A0097B047C1
:10AB800007B0F0BD0A4B10B5984207D1012200234F
:10AB900052420A808B708A808B7110BDFFF73CFF98
:10ABA0000028FAD001235B42038000238370F4E77E
:10ABB000FFFF0000F8B5050001290AD1134E00245B
:10ABC0003388F227AB4219D028001149FFF7DAFF8A
:10ABD00006E0022904D10139FDF73EFF0028EDD03F
:10ABE000F8BD3B0063437268D018D35A002B09D0DC
:10ABF0003A00002100F034FD0134E4B2054B1B782B
:10AC0000A342EED801235B423380DDE7086BFF1FD0
:10AC10002068FF1F066BFF1F10B5FFF7FDFE030046
:10AC20000020834200D0987810BD0000F0B589B0B4
:10AC30001C000EAB80CB03901E8810AB1B780492D7
:10AC400002930B7A0D00DB0616D42B780593022BAA
:10AC500024D00498FFF7D2FE002812D003689C4647
:10AC6000002B0ED0029B2200019329003B0064467A
:10AC700003980096A04705E00498FFF7BFFE002860
:10AC800002D10E2009B0F0BD8368002BF9D00A2252
:10AC90002900039898470028D7D0F3E76B685878C5
:10ACA0001A786B4B000210439842D2D8043B98426A
:10ACB00010D2684B984242D015D8674BC018012873
:10ACC000C7D80B20002EDDD1EB681A7859683A807E
:10ACD000200028E0614BC018032800D979E000F07B
:10ACE0004FFF846A789E5E4B9842B2D10B20002EB3
:10ACF000C8D101233B80EB6831001B782370688941
:10AD0000013080B2FCF790FF3A88031E0ED0017824
:10AD100002328A183A80428962704289120AA2700D
:10AD200059680278E01C00F03BFD06E004323A80EE
:10AD300031000422601C00F093FC0020A2E70B20ED
:10AD4000002E9FD1EB6807A91E8804233B80330A9D
:10AD5000300026706370FCF767FF051E28D004AB37
:10AD60009A890E2304A95B183E49C668FCF7D0FFF8
:10AD700000280BD12B783C486A680599FBF786FBC5
:10AD8000002803D1012304AA5B42D3813278022A2E
:10AD900006D17168201D00F003FD3B8802333B8023
:10ADA0000E2304AA9B181B88A3701B0AE370C4E738
:10ADB00004ABDE81F4E70B20002E00D062E7E968E7
:10ADC0000398FFF729FF02233B802070000A607080
:10ADD000B3E70B20002E00D054E70222EB681B885B
:10ADE0003A8023701B0A6370A7E7E86800F0E8FE6A
:10ADF000C2B203000720B24200D243E70DD002994D
:10AE0000DBB27118994202DB921BD3B20293029B10
:10AE1000E9681A003B8089195AE70023F6E70B20FE
:10AE2000002E00D02EE70722EB683A801A782270B5
:10AE30005A7862705A88A2705A88120AE2701A7997
:10AE40002271DA886271DB881B0AA37175E7C0463C
:10AE5000042900000228000000D8FFFFFFD6FFFFF2
:10AE600003280000FFFF0000A8BE0011F0B58DB060
:10AE70006B460020089120229B5E83423DDAA64B60
:10AE8000187800F0BDFC071E32D00378B02B2CD10F
:10AE90000079023816281FD800F04AFD17001E005E
:10AEA0001E001E0031001E0096001E001D011E0027
:10AEB00052011E0073011E00CD011E0050021E0033
:10AEC0001E001E008E021E00E302944B94491B8854
:10AED00078880B80FBF71AF83800FCF79BFF914B42
:10AEE0001B68002B01D038009847380000F0B0FEF6
:10AEF0008020089B0002434018000DB0F0BDEE22F8
:10AF00000021874800F0ACFB0BAA3B7B798938898C
:10AF100000923A000D32FCF79FFD0400804B1B7835
:10AF2000002C3FD146E0804B788805937F4B410051
:10AF3000CB5A0BAE073BDBB232880293002301935E
:10AF40007B4B210006930093059BFFF76FFE744D2A
:10AF5000002810D1069B3A8A1B889A420BD13800F0
:10AF60000599123000F074FD002804D02B78628916
:10AF70009B00EB185A80162306A81B183288200065
:10AF80007989FCF7C5FE2B7804009A00AA1851882D
:10AF90000029C3D00133DBB22B70002807D006A9EB
:10AFA000C98A9180634A12889A42BCD802E0012182
:10AFB00049429180002B04D059497888FAF7DAFF8A
:10AFC0008AE73E890A2479E000253E89574B06939B
:10AFD0007B88069A5B009B5A033B9D4202DB002D57
:10AFE000F0D05BE0162206A812183B7B798900920C
:10AFF0003A0030000D32FCF72FFD0590002858D0A4
:10B000004689017A7888FCF7F1FC041E44D1464B4E
:10B0100078880793069B4100C95A454B0439C9B249
:10B0200006AAD28A06930291019400930599079B80
:10B03000FFF7FCFD041E2FD1069B39491A88931C8B
:10B04000002D26D14B807988384B4900CB5A5119B5
:10B05000033B8B4220DD059B31485B8941190B7115
:10B06000A91C0135C9B2EDB2059145191B0A2B7116
:10B07000059B2D490433181800F092FB2C4B059AC0
:10B080001B88D318DDB22C4B9E4205D00136B6B2D8
:10B090009CE749889942D6D0002D0CD0204C28003E
:10B0A000618800F05DFB207021007888FAF772FF5C
:10B0B00012E7059CF0E7002C00D183E77B78142B86
:10B0C00000D109E716493B794E800B700C717888E6
:10B0D000FAF712FF00E7162406ABE41821003889BE
:10B0E000FCF7A2FD011E00D1B7E1788822880F4C41
:10B0F00045002C5B0A4D013CE4B2029400240F4B46
:10B1000001940095FFF792FD041E00D014E1290080
:10B110007888FAF74FFFDFE6106BFF1FE042FF1F52
:10B120002868FF1F1C68FF1F1C69FF1F5864FF1F52
:10B130000C6AFF1FDE42FF1FFFFF00002A68FF1F8F
:10B14000162406ABE41821003889FCF76DFD011EBA
:10B1500000D182E178882288AE4C45002C5BAE4D50
:10B16000013CE4B202947C89AC4B01940095FFF75A
:10B170005DFD041E00D0DFE029007888FAF724FF87
:10B18000AAE60025A44B1D803B00F6331B78A24A9B
:10B1900078880792AB4208D99E4B1288069306998D
:10B1A00043005B5A013B9A4203DB0799FAF716FF0B
:10B1B00092E616246B00FB18059306ABE418059B7A
:10B1C00021001889FCF730FD011E03D1059B0124E5
:10B1D0001E8973E77888924B2288069C0993430066
:10B1E0001B5B904E013BDBB2029300230096019360
:10B1F000099BFFF71BFD041E02D0059B1E895DE71E
:10B200007B88069A5B009B5A079A1088328812182E
:10B21000934202DC1B1A013B33807F4C02303288A0
:10B220000999001900F0BCFA2388328801359B186F
:10B230002380EDB2A8E70BAA3B7B7989388900927D
:10B240003A000D32FCF708FC00250590059B002B09
:10B2500004D10A24002D00D16EE060E0059B7888BF
:10B26000197AFCF7C3FB0100041E63D1694C6C4BD7
:10B27000788806940993069B4400E45A694B063C7F
:10B28000E4B20BAE328807930294019100930599C2
:10B29000099BFFF7CBFC041E4CD1079B5E491B8822
:10B2A0001A1D002D30D14A80059B5B4C5A896319C9
:10B2B0001A716B1C9BB2E318120A1A71162306A8A6
:10B2C00032881B1879890598FCF722FDFF21AA1CFA
:10B2D0002E1D03350B00059092B2B6B2ADB2002818
:10B2E00003D006ABDB8AD9B21B0AA218651911710B
:10B2F0002B714C4D301D2A884949201800F050FA16
:10B300002B88F618B5B2A1E74988914207D17A880F
:10B3100006995200525AEB18053A9A42C4DC3E4C48
:10B320002800618800F0D4FB207021007888FAF7AB
:10B330005FFED1E5002DF2D13E89BFE6162606ABB1
:10B34000F61831003889FCF76FFC3D000400FA352F
:10B3500000282DD0037A9B060CD400227B893989E2
:10B36000788800923A000C32FFF7E8FB041E10D0F8
:10B370003E8915E03088FFF741FB00281AD083682A
:10B38000002B17D02100122278889847041EE4D0A1
:10B39000EEE72B78002B02D17888FAF739FE0026E9
:10B3A0002B78002B00D097E5002C00D194E585E6A2
:10B3B0000124DDE70E24DBE7162506ABED18290096
:10B3C0003889FCF731FC041E47D0037A9B0611D460
:10B3D000154A7B881188994203D01448814207D1CD
:10B3E0001380134BF2261D780023D9B2A94221D332
:10B3F0000924A1E72888FFF701FB00282FD08368E4
:10B40000002B2CD02100122278889847041EDFD010
:10B4100092E7C0465864FF1F2868FF1F2A68FF1F75
:10B420001C69FF1F0C6AFF1F086BFF1FFFFF000056
:10B43000066BFF1F31005943546801336018615A8D
:10B440000029D2D13C0008342100F22200F0A8F9F2
:10B4500021007888FAF7E4FD3EE501246CE70E242C
:10B460006AE71D4B1A887B889A4231D07888FAF7B0
:10B47000E1FD31E5F223059851684343CD18C95ADF
:10B4800000291FD03B7A012B0BD16C88AB887888C0
:10B49000AA1D0094FFF752FB041E02D000233B724A
:10B4A0002E88F2220021280000F0DAF800232B80F9
:10B4B000059B0133DBB20593084B05991B78064ABF
:10B4C0008B42D7D801235B421380002CCED0F5E508
:10B4D000002634000596EFE7086BFF1F066BFF1F81
:10B4E00070B504000E001500FFF796FA031E08D190
:10B4F00031000548FFF790FA03001120002B02D01D
:10B500001C8000209D7070BDFFFF0000F8B50B4F40
:10B5100006003B780D001400FF2B0ED00A2000F02F
:10B52000FFF9011E09D0B123038000234680037177
:10B53000C5800481387800F0B3FAF8BD3544FF1FA8
:10B54000F7B50F0008A90600088809A90B24098887
:10B55000002821D10234022B1ED1557813782D02F8
:10B560001D432B008B4301937334002B14D1FB68D4
:10B57000300019000093FFF74FFB019C85420BD070
:10B580002A0030000099FFF7ABFF041E04D12A0007
:10B5900030007989FFF7BAFF2000FEBDF0B50E78C4
:10B5A00085B003900AA805880120022E0DD14C68B1
:10B5B0002778647824023C43054FBC4205D10398A8
:10B5C000DBB201960095FFF7BBFF05B0F0BDC046AA
:10B5D00002290000034B10B51B68002B00D09847D0
:10B5E000FEE7C046146BFF1F07B501A8FFF7F2FF87
:10B5F000044A05480021121A00F0BAF9F8F7FAF8DF
:10B60000FEE7C046186BFF1F3844FF1F0000000014
:10B6100001B40248844601BC604700BF9D35FF1F4E
:10B6200001B40248844601BC604700BF4550000099
:10B6300001B40248844601BC604700BF3D180000C9
:10B6400001B40248844601BC604700BF193BFF1F9C
:10B6500001B40248844601BC604700BF0132FF1FAD
:10B6600001B40248844601BC604700BF154D01008B
:10B6700001B40248844601BC604700BFEDA500004C
:10B6800001B40248844601BC604700BF456B01001D
:10B6900001B40248844601BC604700BF85520100E6
:10B6A00001B40248844601BC604700BFA9460100BE
:10B6B00001B40248844601BC604700BF5147010005
:10B6C00001B40248844601BC604700BFC135FF1F7A
:10B6D00001B40248844601BC604700BF35550000F4
:10B6E00001B40248844601BC604700BF59520100C2
:10B6F00001B40248844601BC604700BF29510100E3
:10B7000001B40248844601BC604700BF7139FF1F85
:10B7100001B40248844601BC604700BFC51D00005B
:10B7200001B40248844601BC604700BF4D1F0000C1
:10B7300001B40248844601BC604700BF2932FF1FA4
:10B7400001B40248844601BC604700BFF94C0100C7
:10B7500001B40248844601BC604700BF1930FF1F96
:10B7600001B40248844601BC604700BF350E0000AA
:10B7700001B40248844601BC604700BFDD66010099
:10B7800001B40248844601BC604700BFC9260000DE
:10B7900001B40248844601BC604700BFC5210000D7
:10B7A00001B40248844601BC604700BFE94C010077
:10B7B00001B40248844601BC604700BF5118FF1F16
:10B7C00001B40248844601BC604700BF75A900006F
:10B7D00001B40248844601BC604700BF156B0100FC
:10B7E00001B40248844601BC604700BF8B5201008F
:10B7F00001B40248844601BC604700BFC94A010049
:10B8000001B40248844601BC604700BFF54E010008
:10B8100001B40248844601BC604700BF311B0000F0
:10B8200001B40248844601BC604700BFD92FFF1F06
:10B8300001B40248844601BC604700BF090E000005
:10B8400001B40248844601BC604700BF0539FF1FB0
:10B8500001B40248844601BC604700BFD9490100D9
:10B8600001B40248844601BC604700BF3D4B010063
:10B8700001B40248844601BC604700BF01240000B7
:10B8800001B40248844601BC604700BFC9A900005A
:10B8900001B40248844601BC604700BF5D17000048
:10B8A00001B40248844601BC604700BFED4A010074
:10B8B00001B40248844601BC604700BFC12FFF1F8E
:10B8C00001B40248844601BC604700BF792DFF1FC8
:10B8D00001B40248844601BC604700BFED39FF1F38
:10B8E00001B40248844601BC604700BF1D4B010003
:10B8F00001B40248844601BC604700BFE54800002F
:10B9000001B40248844601BC604700BF79180000BA
:10B9100001B40248844601BC604700BF11470100E2
:10B9200001B40248844601BC604700BF1D4D0100C0
:10B9300001B40248844601BC604700BF413BFF1F81
:10B9400001B40248844601BC604700BF017F00008B
:10B9500001B40248844601BC604700BFB54C0100F9
:10B9600001B40248844601BC604700BF25260000A0
:10B9700001B40248844601BC604700BFB70E000016
:10B9800001B40248844601BC604700BF6130FF1F1C
:10B9900001B40248844601BC604700BFF30E0000BA
:10B9A00001B40248844601BC604700BFD91B0000B7
:10B9B00001B40248844601BC604700BF65710100C4
:10B9C00001B40248844601BC604700BF056A00001C
:10B9D00001B40248844601BC604700BF4D38FF1FD8
:10B9E00001B40248844601BC604700BF8D120000CC
:10B9F00001B40248844601BC604700BF0D520100FB
:10BA000001B40248844601BC604700BF4537FF1FB0
:10BA100001B40248844601BC604700BF091B000016
:10BA200001B40248844601BC604700BFA54F010035
:10BA300001B40248844601BC604700BFE117000022
:10BA400001B40248844601BC604700BF7D18FF1F57
:10BA500001B40248844601BC604700BFCD4C0100E0
:10BA600001B40248844601BC604700BFC52DFF1FDA
:10BA700001B40248844601BC604700BF4551010043
:10BA800001B40248844601BC604700BF5933FF1F20
:10BA900001B40248844601BC604700BF6DBC000091
:10BAA00001B40248844601BC604700BF594F010001
:10BAB00001B40248844601BC604700BF055E000037
:10BAC00001B40248844601BC604700BF291C000045
:10BAD00001B40248844601BC604700BF090E000063
:10BAE00001B40248844601BC604700BF350E000027
:10BAF00001B40248844601BC604700BF691F0000D2
:10BB000001B40248844601BC604700BF810E0000BA
:10BB100001B40248844601BC604700BF55220000C2
:10BB200001B40248844601BC604700BFE928000018
:10BB300001B40248844601BC604700BFC56D0100E6
:10BB400001B40248844601BC604700BF9DA90000C3
:10BB500001B40248844601BC604700BF2146010091
:10BB600001B40248844601BC604700BF851F000045
:10BB700001B40248844601BC604700BF9136FF1FF4
:10BB800001B40248844601BC604700BF2D3BFF1F43
:10BB900001B40248844601BC604700BFD91AFF1FA8
:10BBA00001B40248844601BC604700BF9135FF1FC5
:10BBB00001B40248844601BC604700BF2124000054
:10BBC00001B40248844601BC604700BFDD52010059
:10BBD00001B40248844601BC604700BF8538FF1F9E
:10BBE00001B40248844601BC604700BFADAE00000E
:10BBF00001B40248844601BC604700BFB352010053
:10BC000001B40248844601BC604700BF014C0100FA
:10BC100001B40248844601BC604700BF5549010099
:10BC200001B40248844601BC604700BFB14E000029
:10BC300001B40248844601BC604700BF51250000A2
:10BC400001B40248844601BC604700BFC538FF1FED
:10BC500001B40248844601BC604700BF434D010067
:10BC600001B40248844601BC604700BF3938FF1F59
:10BC700001B40248844601BC604700BF193AFF1F67
:10BC80000001010302000303040305020602070288
:10BC9000080209020A030B030C020D000E030F0336
:10BCA000100311001300140315001600C53B00110A
:10BCB000F93B00110000000002000000C2BC0011AE
:10BCC000192A0F180A000000F1590000FD24000095
:10BCD000414601006580001179A00011CD7400116A
:10BCE000697E0011315300116DAE0011994F0011A2
:10BCF000D53D0011053F00110000000016160000A0
:10BD0000020000000CBD0011F4FFF3FFD2FC0000A4
:10BD100045400011000000000000000054757961EA
:10BD20000042312E35003030313900676974687552
:10BD3000622E636F6D2F70767678005448303546EA
:10BD4000000000000200000058BD0011292A282A26
:10BD5000272A262A252A242A0A180000E20400009D
:10BD60007102000078EC0000744000001027000011
:10BD700060F0000006640000204E0000000000009B
:10BD8000050000001F501D00023CB4000001190016
:10BD900015000000A102000030313233343536374F
:10BDA00038394142434445460000000035570011F0
:10BDB000895700110000000002000000C4BD0011FE
:10BDC0006F2A6E2A1A18EAD8BC80F0FC60000000C6
:10BDD00000000000000000F505D39727B6F615F720
:10BDE000B777E6F0C7F27200000001A00000000083
:10BDF0006410B71DC8206E3BAC30D9269041DC766C
:10BE0000F4516B6B5861B24D3C7105502083B8ED15
:10BE100044930FF0E8A3D6D68CB361CBB0C2649B39
:10BE2000D4D2D38678E20AA01CF2BDBDFB349B5F5E
:10BE3000800000800010000000000000CF600011B2
:10BE400059770011F3600011617B001177610011D7
:10BE5000377B0011ED6100110D7B00113F62001175
:10BE6000D57C0011A7620011D57C0011D9620011A8
:10BE70008F7C0011ED610011C57A0011656200111F
:10BE80006D7C001100000000000000004B630011F9
:10BE90006D7C0011AD63001171770011052A042A31
:10BEA000012A002A02290328012800280118001865
:10BEB00000000000000000000000000000000087FB
:10BEC0000101020102010102010203030401030155
:10BED000010101010303020103000D000E00100027
:10BEE000110013001401070108010A010B011C01D4
:10BEF0001D02040205020702080219021A021C02AE
:10BF00001D030103020317000201000504000807D6
:10BF1000000B0A001716001D1C0102010105040197
:10BF20000E0D011110011413011716011A19020246
:10BF300001020B0A020E0D02111002141302171651
:10BF4000030504030807030B0A030E0D0001020397
:10BF500007090A0B0E0F101112141718191A1B1FBC
:10BF600020212200B5A7001171A8001100000000D7
:10BF700002000000AEBE0011000000009DB50011DF
:0CBF80000000000002000000ACBE001138
:020000041FFFDC
:10000000000000003D3D0011C8BC0011C4BC00113F
:100010004461FF1F0000000000000000000000001D
:1000200000000000000000000000000000000000D0
:1000300000000000000000000000000000000000C0
:1000400000000000000000000000000000000000B0
:1000500000000000000000000000000000000000A0
:100060000000000000000000000000000000000090
:100070000000000000000000000000000000000080
:100080000000000000000000000000000000000070
:100090000000000000000000000000000000000060
:1000A0000000000000000000000000000000000050
:1000B0000000000000000000000000000000000040
:1000C0000000000000000000000000000000000030
:1000D0000000000000000000000000000000000020
:1000E0000000000000000000000000000000000010
:1000F0000000000000000000000000000000000000
:1001000000000000000000000000000000000000EF
:1001100000000000000000000000000000000000DF
:1001200000000000000000000000000000000000CF
:1001300000000000000000000000000000000000BF
:1001400000000000000000000000000000000000AF
:10015000000000000000000000000000000000009F
:10016000000000000000000000000000000000008F
:10017000000000000000000000000000000000007F
:10018000000000000000000000000000000000006F
:100190004D32FF1FAD30FF1FC1660100000000009F
:1001A000000000000000000000000000000000004F
:1001B000000000000000000000000000000000003F
:1001C000000000000000000000000000000000002F
:1001D000000000000000000000000000000000001F
:1001E000000000000000000000000000000000000F
:1001F00000000000000000000000000000000000FF
:1002000000000000000000000000000000000000EE
:1002100000000000000000000000000000000000DE
:1002200000000000000000000000000000000000CE
:1002300000000000000000000000000000000000BE
:1002400000000000000000000000000000000000AE
:10025000000000000000000000000000000000009E
:10026000000000000000000000000000000000008E
:10027000000000000000000000000000000000007E
:10028000000000000000000000000000000000006E
:10029000000000000000000000000000000000005E
:1002A000000000000000000000000000000000004E
:1002B000000000000000000000000000000000003E
:1002C000000000000000000000000000000000002E
:1002D000000000000000000000000000000000001E
:1002E000000000000000000000000000000000000E
:1002F00000000000000000000000000000000000FE
:1003000000000000000000000000000000000000ED
:1003100000000000000000000000000000000000DD
:1003200000000000000000000000000000000000CD
:1003300000000000000000000000000000000000BD
:1003400000000000000000000000000000000000AD
:10035000000000000000000000000000000000009D
:10036000000000000000000000000000000000008D
:10037000E9B50011000000000000000000000000CE
:10038000000000000000000000000000000000006D
:10039000000000000000000000000000000000005D
:1003A000000000000000000000000000591AFF1FBC
:1003B000000000000000000000000000000000003D
:1003C000000000000000000000000000000000002D
:1003D000000000000000000000000000000000001D
:1003E000000000000000000000000000000000000D
:1003F00000000000000000000000000000000000FD
:08183800206FFF1F4118FF1F84
:10184000024981F3088802F04FFB0000206FFF1F60
:1018500010B502F0B1F9072804D0122808D00228E8
:1018600008D010BD044A0420136B01331363F8E75A
:101870000220F6E71420F4E70065FF1FF8B5070023
:101880000C0026002500503630785135002804D150
:101890000300287058342370F8BD2978CA00481E08
:1018A0008141A3183800A25C5B68C9B2FFF7D0FF82
:1018B00000280DD12B78DA00A218013350602B706C
:1018C0003378044A013B3370136A01331362D8E75B
:1018D0000123DFE70065FF1F5C234343074910B581
:1018E000C9180B0058331B78012B05D1FFF7C6FF31
:1018F000034A936A0133936210BDC0463465FF1FEB
:101900000065FF1F10B502F0C7FA064A0121130057
:1019100010CB4942D967044B136002F09DFB2000B5
:1019200010BDC04600E100E01000100010B504003A
:1019300002F0B2FA024B1C6002F08EFB10BDC046F2
:1019400000E100E0431E5A425341A022F0B5D2010B
:101950005B421340154D164A40019B182A18127E0F
:101960008BB00191002A1BD01A000832D46F0022DC
:10197000E6B206AFE4B294420EDC2818C369002B2D
:1019800008D0019902AA117106AA049202AA16733C
:1019900003A898470BB0F0BD1978B9540132EAE7B3
:1019A0001A7D1A7806AB01261A70E6E7C067FF1F9A
:1019B00000400040F0B5254B04004001C25C85B0FA
:1019C000002A2BD01A18117E002927D0917E0029D9
:1019D00024D01179022921D11689D788D168F51B25
:1019E000ADB22A1C102D00D9102292B2BE4217D1DE
:1019F0001818012303710023C269C38003819A422E
:101A000006D06846032103730171029301A8904731
:101A10000820002C00D0192001F0FEFA05B0F0BD1E
:101A2000013C65426C41A0256442ED012C40084D0B
:101A30001B186419074D0633013A92B2AA42EDD041
:101A40001888461C1E80085C2070F5E7C067FF1FE1
:101A500000400040FFFF00000F220E4B10B59868B9
:101A6000104002380A280BD802F060F80D0A0B0A61
:101A70000A110A0A0A0A060002210020FFF762FF83
:101A800010BD0121F9E70020FFF794FFF8E7DB6FB5
:101A9000F6E7C046004000400F220E4B10B5986894
:101AA000104002380A280BD802F040F80E0A0B0A40
:101AB0000A120A0A0A0A060002210120FFF742FF61
:101AC00010BD01210800F9E70120FFF773FFF7E7D8
:101AD000DB6FF5E70090004013B5334C2378072BFC
:101AE0003DD8324B1A78324B002A39D180221968FE
:101AF00052020A431A60252001F0C4FE20232D4A19
:101B000011680B43802113606B460422C9050868E5
:101B10000733104228D080210422C905C86810422A
:101B20002ED080212020C905CA688243CA601422B1
:101B30001A701A78002A2FD18021C905C86820326E
:101B40000243CA6014221A701A78002A28D11A4B4C
:101B50001A7D22785A601D221A705932DA6013BD3C
:101B60001A6816490A40C5E7086802430A60142249
:101B70001A701A78002ACED01A78013AD2B2F7E752
:101B8000C8680243CA6014221A7019784A1ED2B279
:101B90001A700029F9D1C4E71A78013AD2B2C7E71E
:101BA0001A78013AD2B2CEE77043FF1F3844FF1FC4
:101BB0003CF000406843FF1F00200040FFFFFEFF95
:101BC000564B70B51B68012B03D1554A936D0133F9
:101BD000936502F0D1F9534B534A1860534B544C60
:101BE0001A600123534A1360534A13602378002B71
:101BF00006D006225149524802F0DEF80023237035
:101C0000504A514B10681B78C1B2002B0ED14F4C7B
:101C1000C0B223785BB2002B4FDB237824785BB211
:101C200064B21B0424021B191B1813600B1C5029DF
:101C30004ED95023464A47491078DBB2FF2202288A
:101C40004BD10868444C454D267890432A789642FB
:101C500054D9227824782E78023B5D10A31B6B4365
:101C60005201D31A10335B111843086002F094F844
:101C7000031F012B45D83A4B1B78002B06D0394B5C
:101C80001B78002B02D0002002F036F9A122364B3F
:101C900092009978354B4A431B689B188322920027
:101CA0009B181B78033B012B03D8AF20400001F0A9
:101CB000FBFF01222E4BDA8270BD237824785BB2C1
:101CC00064B2FF33FF341B0424021B190138ABE755
:101CD000CAB2022AAED20223ACE70868254C264DD0
:101CE000267890432A78964208D9227824782D784D
:101CF000023B5B10641B63435201B2E72378DBB203
:101D0000B2E70228D5D11D4B1B78013B022B03D92A
:101D10001B4B1B78022BCCD16C20C8E79809FF1F06
:101D2000FC0FFF1F3864FF1FFF3F0000141003402B
:101D30003C64FF1F0C10034000100340D50BFF1F35
:101D40007211FF1FB40003408C09FF1F680AFF1FB8
:101D5000490AFF1F94000340460AFF1F470AFF1F5E
:101D6000F908FF1F2209FF1F300DFF1F3409FF1F55
:101D7000BC0BFF1F440AFF1F450AFF1F1C09FF1F62
:101D80002309FF1F10B502F017F90022014B1A803A
:101D900010BDC0463664FF1F10B502F045F8A12102
:101DA000054A89009478054A61431268044B521829
:101DB000528C1A8010BDC046300DFF1F3409FF1F22
:101DC0003664FF1F10B50D4B0D4A9978A1239B0077
:101DD0004B431268D218531DD97F0A4B1B88994276
:101DE00009D2441C07D0C82805D0D2695B1A5A43CF
:101DF000054B5343C01802F017F910BD300DFF1FFB
:101E00003409FF1F3664FF1F7102000070B5244DB6
:101E10002B68002B28D002F0F7F82B68D8402B68ED
:101E20000400002B27D002F06FF82B68D8401D4B20
:101E30001D4A9978A1239B004B431268D118D25CAC
:101E400091239B00002A20D0CA580132CA50174B58
:101E500017491B680868834214D3D23B181A012A19
:101E60001AD0144B186070BD02F0CEF8124B1968EE
:101E700001F072FFD3E702F047F80F4B196801F049
:101E80006BFFD4E70D495B18E8E7CA500C4B1B68A1
:101E9000DB68E418201AE4E7F530FF30E1E7C046DC
:101EA0001C08FF1F300DFF1F3409FF1F9C09FF1F77
:101EB0003864FF1FA009FF1F1808FF1F2DFF3F00F8
:101EC0004064FF1F70B504000D00282916D10300DF
:101ED000A433C2881B889B1A0B4A9BB293420DD92C
:101EE00006006A3605223100653001F03DFE00280B
:101EF00004D13100200002F07FF870BD29002000DD
:101F000001F00AFFF9E7C046FE7F0000F8B50500C2
:101F1000012001F0B9FF134CA36AA26A9342FBD1DE
:101F2000114E336002F018F81049030008601048A1
:101F3000426894460F4A17680022BC4501D24268A5
:101F4000BA1A0D4802603268AD18A422E562606AD0
:101F5000520302436262094A1278002A01D00F3B01
:101F60000B60F8BD00F00040340AFF1FE408FF1FBB
:101F700028100040180AFF1F1C0AFF1F1C09FF1F22
:101F800070B580241025E405A3682B43A36001F0FD
:101F90005BFEA368AB43A36070BD0000F7B51600FD
:101FA00080221C001023D2050191916805000B438B
:101FB000936000225A4BD7301A6001F045FF9D23F1
:101FC0002A002F009B00EB58CA3201210092FC37F7
:101FD000002B01D00021009A386801F0B5FF2900DC
:101FE000009BCB311A784F4BD3351A604B780A7867
:101FF0001B0213438A7812041A43CB781B0613433F
:10200000494A1BBA13604B790A791B0213438A7938
:1020100012041A43CB7931001B061343434A1BBAFF
:1020200013606B782A781B021343AA7812041A43B0
:10203000EB781B0613433E4A1BBA1360019A330226
:1020400013433C4A13603C4B22001B1B9C46032954
:102050003DDCB3089A0013005142B21A032A46D15C
:10206000354AE018511A827840781204000202437F
:10207000E05C043302430A600022FF2B4BDDF022B8
:102080002E4B12011A600F222D4B1A602D4A136835
:10209000002BFCD00023224A27491360091B321D64
:1020A0000B191B68043A180A23706070180C1B0E79
:1020B000A070E3700434002AF2DC802210213B6817
:1020C000D20501333B6093688B439360F7BD634651
:1020D000D578981893782D061B042B43157804396E
:1020E0002B43557804322D022B430360AFE7022ABD
:1020F0000AD1114AE05C511AE218527812020243E6
:102100000A6004339BB2B7E7012AB5D10A4A521AD2
:10211000E15C1160F5E7084959180A600433ACE73F
:10212000000004403C0004403800044034000440F7
:10213000300004400C00044000010440040004404E
:102140001000044014000440F7B5150080221C0064
:102150001023D2050091916807000B439360002380
:10216000654AD730136001F06FFE9D233E009B004F
:10217000F9583B00CA363200FC33002900D07FE01A
:10218000586801F0E1FE390032785C4BCB311A60BF
:102190004B780A781B0213438A78AC4612041A4320
:1021A000CB78281D1B061343554A1BBA13604B7985
:1021B0000A791B0213438A7912041A43CB791B064E
:1021C0001343504A1BBA13604B7A0A7A1B0213431B
:1021D0008A7A12041A43CB7A21001B0613434A4A17
:1021E0001BBA1360009A2B021343484A1360220063
:1021F000474B1B1B0093009BCE785B1801938B7899
:1022000036061B0433430E78043833434E780431CA
:1022100036023343019E33600328ECDC0321A80817
:10222000431C9B002940800003292BD13849E51825
:102230005E18A9786D78E35C09042D0229431943DF
:102240003160030008330021FF2B2DDD314B324973
:1022500019600F21314B1960012327490B60304B66
:1022600019680029FCD006211B680B40042B20D0E4
:1022700080220020D20593680A318B439360FEBD13
:1022800001217DE7022908D121495D18E11849782B
:10229000E35C090219432960D3E70129D3D11C4922
:1022A0005918E35C0B60CCE7194818180160043337
:1022B000CAE7002310490B606346002B0CDC3B008F
:1022C000FC335A68102101325A608022D20593688B
:1022D00001208B439360D2E7009B9B181B68190A6F
:1022E00013705170190C1B0ED37004235B42917054
:1022F0009C440432E0E7C046000004403C00044037
:102300003800044034000440300004400C00044015
:102310000001044004000440080F000010000440C5
:102320001400044070B5061E19D002225A4B9B7946
:102330009343012B13D1594B1A78FF2A0FD15A78A6
:10234000FF2A0CD19A78FF2A09D1DA78FF2A06D120
:102350001A79FF2A03D15B79FF2B00D199E0504B0A
:102360000C201A78012A08D000224E4D1A702978C4
:102370000B00093B042B01D8212070BD4B1F012B02
:10238000FAD9454CA37B042B00D982E0A279032A19
:1023900000D97EE09A1ED2B2012A02D860881F2896
:1023A00077D9002E56D0012E73D1A0880128E3D012
:1023B000002907D1581E032803D801F0B7FB1217D4
:1023C00015122E702978481E032811D80025364B87
:1023D0001D602823237501F097FCA84227D0A58013
:1023E000CAE702212970EDE70421FBE70321F9E7A1
:1023F00007390129C0D82D490968C96A8906BBD5A2
:102400002B4908780028B7D1012A01D9002BB3D174
:1024100002230B708021274D2633890128782375EC
:1024200001F002FC80212878890101F0F5FD0123EB
:10243000A380214B1B78002B0AD0FA2280211F4B4E
:1024400092001B8809025A431A4B187801F0A4FB2A
:10245000002092E701F020FD2B78A680073B012B9E
:1024600003D917482E7001F09FFC114B114C1A78BC
:10247000002A06D080210022207889011A7001F0FC
:10248000D3FB01F0E9FD80212078090201F0CCFBAB
:10249000DEE7122071E7C046A60BFF1F6B09FF1F86
:1024A0001A09FF1F1C09FF1F4809FF1F4064FF1F77
:1024B0002309FF1F1B09FF1F2109FF1F2C09FF1FF5
:1024C0000010004010B5002901D001F0D5FC10BD6E
:1024D000F7B5604B01919978A1239B004B435E4A6D
:1024E000060014681022E418D6235B00E058362357
:1024F000FF33E35C00279343222B41D1574B0F3A24
:102500001A600760012501F097FD019B1880E82300
:102510005B00E35C002B01D0B34258DD0023504F39
:10252000FB70AD33FF33E3581A68002A03D09B8851
:10253000DB439B071DD03823FF33E35C002B18D00F
:102540009B235B00E35C002B13D1D133FF33E35CAF
:10255000B3420EDAA4235B00E15AE018090A023103
:1025600001F07AFC23000122FE33013E01351A8777
:10257000FA70E8235B00E35C002B2AD0A8B2FEBD12
:1025800003683D00002BBED081880430090A023167
:1025900001F062FCD6235B00E3581F60B2E7230022
:1025A000B133BA00FF339858013781880430090AE3
:1025B000023101F051FCE8235B00E35CBB42EEDC3E
:1025C000E822F61AED1800235200A354A6E70027CC
:1025D000F1E7200001F0E0FC00281FD0002E1DDDF7
:1025E0007319882647190193B600200001F04CFBAF
:1025F0005A30800020184068013581880430090A6B
:10260000023101F029FC200001F04EFCA3590133F6
:10261000A351BD4202D0019B9D42E6D1114BE35C28
:10262000002BABD095239B00E35C002BA6D00E4B78
:10263000E15A0029A2D00D4AA35C994202D9013384
:10264000A3549BE700231A212000A35401F09CFA15
:1026500094E7C046300DFF1F3409FF1F00140340EC
:10266000E010FF1F5A020000720200005E0200002C
:102670000D4970B54A6E0D4CD2038B69D20BA24244
:1026800006D80B4D0224AA4204D901F0ADFA70BD60
:1026900002246442E21815007E2425402242F4D030
:1026A000A3432B438B61F0E700F000400A200000B9
:1026B000FC1C0000F8B51D4B1D4F1A78002A10D1E4
:1026C000BA7B002A02D101321A7003E0032AFAD041
:1026D000022AF8D001F018FB00220120154B1A70D5
:1026E000F8BD154B154D1C68154B9E7801232B70BA
:1026F0002878C0B200F0A2FBBB7B002B0BD101F00D
:10270000DBFBA1239B007343E41883239B00E418A5
:1027100023782B70E4E7032B02D101F0A5FBF0E74F
:102720000020022BDCD101F00FFBEAE71C09FF1FA0
:10273000A60BFF1F2309FF1F3409FF1F490AFF1FB4
:10274000300DFF1FF0B587B00EAD2F780FAD2D788F
:102750000593AC46634614000E4D0CAA12782E78F1
:1027600003930D9B009201932200059B029701F0B9
:10277000C3FA2E70012C01D0042C08D18022064906
:102780008B889343054A1278D20113438B8007B09C
:10279000F0BDC0461C09FF1F6C11FF1F7809FF1F09
:1027A0000B001B3B70B504003020E02B0DD813004C
:1027B000E025493BFF3B9BB2ED00AB4205D8034B04
:1027C000200019825A8201F08FFA70BD8410FF1F19
:1027D00010B501F0D1FB054B00205B68052B04D937
:1027E000034A5268D20200D4980810BD001000407D
:1027F000FCE100E070B501F04FFB0D4B1B68FC33B2
:10280000DC691D6AFFF7E4FF6419844204D2094BB6
:1028100001241B68002B07D004220024064B1A70E9
:10282000064A93690133936101F016FC200070BDE4
:102830004064FF1F9809FF1F2309FF1FFC0FFF1FA4
:1028400070B50C4D2B68FC335C6A01F025FBFFF77B
:10285000BFFF2B680025FC339B6AE318834204D238
:10286000054B1B68AB4200D1051B01F0F5FB2800AE
:1028700070BDC0464064FF1F9809FF1FD722044B5C
:1028800092009B5810B5002B00D0984710BDC04651
:102890000000FF1F10B501F0D3F8FFF7EFFF274945
:1028A000274BCA6D274C1A4084235B001343CB652A
:1028B000254B1B68186A01F0E7FA244B244A1A607A
:1028C000244B254A1A60A022244B52001A60244B44
:1028D000187801F031FA2000224901F01DFB002395
:1028E000A3600233A360204B2049236003232048C8
:1028F000A36001F011FB10221E4BFF201A60802202
:1029000052031A60802292031A60802212041A6015
:1029100001F0F2FA012001F047F9FA20400001F03D
:102920007BFA582001F0C0F9134801F065F9012045
:1029300001F0CAF9072001F0FFFA10BD00F00040D5
:1029400000FEFEFF141000404064FF1F0000034023
:102950000180063DBC00034034080000A400034091
:102960004A0AFF1F71020000C3090000FFFF3F0079
:102970002810004000E100E030750000674E336829
:1029800088331B6883F3088801F096F9644A654927
:10299000136800200B401360634B644A1B6893422A
:1029A00000D1A6E001F048FA0221614A13688B4386
:1029B0001360FFF76FFF5F4B5F4C1878C0B201F0F8
:1029C00013FB0023A3600233A3605C4B0120236050
:1029D00001F05AFA0323A36001F00EFA040001F09B
:1029E000CBFA050001F008FA554B186001F00CFA1B
:1029F000544B1968621A531EA14200D21300802260
:102A0000D203934201D39B029B0A3268D16AC90761
:102A100000D471E04C491C0C09689BB24C435943EB
:102A20002402090A641803264849FC3293680A689C
:102A300047489B1A474A0768126847499B18474A04
:102A40009A1833409208DB190A600360042B03D9FB
:102A5000013233400A6003600E684149A619300014
:102A600001F07AF93F4F3E493B68C3183B603000A4
:102A7000019301F0B9F93C4E3068081838493060CC
:102A8000884205D9019B01333B6001F0ADF931600B
:102A900001F08AFA354B1B78002B0DD001F06CFA4F
:102AA000334B621B196812188A4232D24919091B2A
:102AB000091A304801F030FA2F4E337A002B0ED02D
:102AC00001F05AFA621BF1681218914224D949198F
:102AD000091B091A294801F01FFA00233372284BF9
:102AE00083F3088801F078F8002001F0A5F901F0DF
:102AF000A3F801F0A1F95CE7DC0199000234641A43
:102B00005900641A09214B438033CB40A408E418D0
:102B100089E7FA218900CCE71A49DBE74064FF1F07
:102B20001CF00040FFFFC1FF0C0AFF1FB64121034C
:102B300010000040490AFF1F14100040C3090000A4
:102B4000100AFF1F340AFF1F380AFF1F200AFF1F49
:102B5000280AFF1F1C0AFF1F240AFF1FC4090000C8
:102B6000710200006008FF1F2C0AFF1F1C09FF1FD5
:102B7000E408FF1F00100040740BFF1F3C100040D2
:102B800000000020DC050000A022054B92009B58AD
:102B900010B5002B01D0984710BD01F01DFAFBE7DE
:102BA0000000FF1FA122054B92009B5810B5002B7F
:102BB00001D0984710BD01F00FFAFBE70000FF1F9E
:102BC000A222054B92009B5810B5002B01D09847CC
:102BD00010BD01F001FAFBE70000FF1FA322054B27
:102BE00092009B5810B5002B01D0984710BD01F002
:102BF000F3F9FBE70000FF1FA422054B92009B584E
:102C000010B5002B01D0984710BD01F0E5F9FBE7A6
:102C10000000FF1F70B501F0AFF94F4B186000F0D6
:102C2000FBFF0400C30702D401F00EFA70BD0022BE
:102C30004A4B1A604A4B18780138042829D800F00A
:102C400075FF0320181C2400200001F0BDF80128A6
:102C5000ECD0444C2378042B6ED100F07DFF00288B
:102C6000E4D001F039F9582001F01EF80223237056
:102C7000DCE7200001F030F8E9E7200001F07CF803
:102C8000E5E7200001F050F8E1E7200001F09CF9B1
:102C9000DDE701F081F80500012808D1324B1B78EF
:102CA000053B012B03D82000FFF76EFFD1E72D4B2A
:102CB0001B78022B01D0052B20D1022D28D12B4BC4
:102CC0009B7BAB431CD12000FFF76CFF264B187891
:102CD0000128BED16405BCD4244925224B7B034284
:102CE00005D1233A13405A42534126331A000B7D33
:102CF0009342AED9322000F087FFAAE7022D07D118
:102D0000194B1B78052B11D12000FFF759FFDDE788
:102D1000012D0BD1012B03D12000FFF75FFF98E7B6
:102D2000062B03D12000FFF767FF92E7200001F098
:102D300053F9022D8DD1C9E7032B04D10C4B987C9C
:102D400000F042FF72E7072B00D06FE7094B987B3A
:102D500000F012FF6AE7C0469C09FF1F9809FF1F99
:102D60009009FF1F2309FF1F1C09FF1FA60BFF1F50
:102D7000BC0BFF1FD40BFF1FFA210A4B0A4A490064
:102D80001A640A4A5A500A4A04395A50094A083100
:102D90009A64094A5A50094A5C315A50084ADA661C
:102DA0007047C0460000FF1F4527FF1F4128FF1F37
:102DB000F527FF1F2523FF1FB526FF1FC51DFF1F7A
:102DC000991DFF1F10B500F099FE10BDF7B50B0C53
:102DD000FF270122009300233C001E001D009446A3
:102DE000019089B262469A40100008401841361896
:102DF000B6B2FF2F02D1012E00D19FB2009802403F
:102E00001A41AD18ADB2FF2C02D1012D00D19CB2F8
:102E10000133102BE6D10320012E07D1012D04D15F
:102E2000019B2401E4191C700138FEBD102EFCD159
:102E30000238102DF9D00230F7E700008023F7B5F3
:102E40009C46264B264F01932649274A274D284C5E
:102E5000284B02281AD1604638600868264E304058
:102E6000802636033043086001990978002909D18A
:102E70001660224A2A60224A2260E02219689143A1
:102E8000A03A1BE08021C9021160F2E766463E606D
:102E90000F68194E3E408027FF023E430E600199A5
:102EA000097800290DD1176001280ED1154A2A6032
:102EB000154A2260E02219689143C03A0A431A6019
:102EC000F7BD802189021160EEE7E0210F4A02433D
:102ED0002A600F4A22601A688A43F0E74B0AFF1FF4
:102EE000E0000340D800034090000340000003408E
:102EF0005000034040000340FFFFE3FF0280063D17
:102F0000804508220180063D8066082200800698E0
:102F100080550822F8B51E4B80261A680020140040
:102F20003440324232D11A681A4F32431A600122B9
:102F30003B68063093433B6000F0A6FF0122164D2C
:102F40002B681E432E603B680A2613433B60802794
:102F5000BF00124B1B683B4211D1013EF6B2FF2E5F
:102F600009D17E220E4B1C682B68E40B144093435E
:102F700023432B6005E0082000F086FFE9E7002EE0
:102F8000EFD180222B68600893432B60F8BDC046C8
:102F9000C4F000405CF0004018F0004068F00040D1
:102FA00060F0004010B500F067FE01215820034A90
:102FB00000F0DAFEFFF7AEFF10BDC046600AFF1F4B
:102FC00010B578220021034800F066FE00F0DCFE18
:102FD000002010BD4867FF1F70B5040000F05CFFC3
:102FE00000230C200B4A010059438D18515C002925
:102FF0000DD0A14208D1012300246B7000F064FFC2
:1030000001F02AF8200070BD01330A2BEBD1122405
:10301000F6E7C0464867FF1F70B5040000F03CFFAC
:10302000002319001D000D4A1078002806D0A04288
:103030000CD1557001310C320A29F5D1002B0AD17F
:1030400000F0A2FE01F008F8002070BD5078461E86
:10305000B0411B18EEE700F037FFF3E74867FF1FAA
:10306000F7B504000C20002384460E4D01926746FC
:103070005F43E85D7E19A04212D000280BD10A4BB5
:103080009C4662461B7808331370019B70707C5518
:103090007160B360FEBD01330A2BE8D10320F9E76C
:1030A0000720F7E74867FF1F4467FF1F8020F8B538
:1030B000484BC0051B68C1248360474BFF251A6835
:1030C000012313434361454BA4001A68444B40213C
:1030D0001A60444B1A68444B1A60444B1A59AA436D
:1030E0001A51C52292009E58AE4331438026995012
:1030F0009F583F49F6010F403E439E509E588027FF
:103100003602360A3043985080201A5900020A408D
:1031100002431A5104341A59364E3F043240802675
:103120003A431A511A5936061202120A32431A51F8
:1031300008341A5980260A4002431A51C3229200C9
:103140009F58B446AF4337439F509F58294E0F4076
:1031500007439F509F5837408026360437438026C8
:103160009F509F5836063F023F0A37439F50C02268
:103170001F59AF433A431A511A591202120A164301
:10318000C6221E5192009C58AC4365462C439C506D
:103190009C5800250C4020439850C72080001A58A6
:1031A000154C1140C02212020A431A50134B1B78CF
:1031B000DB08AB4201DC0020F8BD2378002B06D0F1
:1031C000A368002B00D0984701350C34EEE712209D
:1031D000F2E7C0466C43FF1F6843FF1FB0F000409A
:1031E0004067FF1FB4F000403C67FF1F00E100E0B4
:1031F000FF00FFFFFFFF00FF4867FF1F4467FF1F3F
:10320000030010B51F2809D8072200201340072407
:1032100004490A78A24313430B7010BD0023062013
:10322000F5E7C0464467FF1F054B06491B780A684F
:1032300005485B0702401B0B134300200B607047DF
:103240004467FF1F1CF00040FFFFC1FF70B50C2555
:10325000FFF7EAFF0A4B1C780A4BE4086543ED18B8
:10326000002C01D1200070BD2B78002B06D06B689C
:10327000002B00D09847013C0C3DF1E71220F2E70B
:103280004467FF1F3C67FF1F1FB5002102220B0090
:1032900001910091052000F047FE02230B490A68C6
:1032A0001A42FCD120230393039B5A1E0392002B46
:1032B000FAD1074A1368002BFCDA0B246C44200077
:1032C000012100F0D1FC207804B010BD90C800406E
:1032D00000C8004013B504000A4B0193019B002B6A
:1032E00001D1112016BDFFF7CFFF23000340044298
:1032F00005D0052000F0C8FD019B013BEDE718005B
:10330000F0E7C046FFFFFF0707B500F0C5FD8022CC
:103310000821D205936A0191002B01D107399162EE
:1033200002210C4A11600199481E01900029FAD12E
:1033300003311160053101910199481E0190002966
:10334000FAD11160002B02D18022D205936200F0E5
:1033500083FE07BD00C00040F0B52D4C89B0237836
:10336000002B4FD1FEF7CEFA02232A4F03903A6882
:103370001A42FCD120230693069B5A1E0692002B6C
:10338000FAD1254E3368002BFCDA0120FFF7A2FFAB
:10339000011E02D0112009B0F0BD030003220190EC
:1033A000009005AD9F2000F0BFFD0321280000F034
:1033B0005BFC02233A681A42FCD120230793079B47
:1033C0005A1E0792002BFAD13368002BFCDA012039
:1033D000FFF780FF0028DDD10398FEF7A7FAAA784F
:1033E0006B7811041B020B4329780B4363601300B5
:1033F000113B0A49052B07D801239340A3600B60BA
:10340000012323700020C6E780231B03F6E7C04694
:103410005443FF1F90C8004000C800409808FF1F99
:103420001E4B30B55A6818781D4B85B0D3185942D9
:103430004B4101210093002300F00EFC194B1A4A66
:1034400002259A6300221A6510325A658022C4212F
:103450009D65164B1648D202DA6789004258154B13
:1034600080241A4080231B041343435064234120CB
:103470000393E40500F006FA402000F003FA6562C9
:10348000039D6B1E0393002DFAD103236362FFF7A4
:103490003BFFA562FFF760FF05B030BD6043FF1F33
:1034A00095FFFEF700C80040050001FF04E100E0C1
:1034B00000E100E0FFFF00FFF0B585B00700FEF778
:1034C00021FA022305002D4C22681A42FCD1202348
:1034D0000093009B5A1E0092002BFAD1284E3368AD
:1034E000002BFCDA0120FFF7F5FE002803D01124A1
:1034F000200005B0F0BD234B2360022322681A424E
:10350000FCD120230193019B5A1E0192002BFAD17A
:103510003368002BFCDA0120FFF7DCFE0028E6D13F
:10352000194B1F60022322681A42FCD12023029308
:10353000029B5A1E0292002BFAD13368002BFCDA50
:103540000120FFF7C7FE0028D1D1104B23600223D2
:1035500022681A42FCD120230393039B5A1E039234
:10356000002BFAD13368002BFCDA0120FFF7B2FE02
:10357000041EBCD12800FEF7D9F9B9E790C8004075
:1035800000C8004001000006A8C8004001800001FA
:1035900010B50020FFF790FF10BD000010B5064BDE
:1035A00018705960FFF73CFF00211320034AFFF712
:1035B00057FD002010BDC0466043FF1F2134FF1F90
:1035C000F0B5040085B003920291FEF79BF98822C2
:1035D00063035B0B52051A438023DB059D6A80233E
:1035E000274F0092BA68002601901B039A420CD91B
:1035F000F82326001B041E401C4206D08022214BCB
:1036000052025E6219680A431A60002D0BD100F065
:1036100043FC02221C4B1A608023DB055A62013AEC
:103620009A6200F019FD0023039A934220D1002DE5
:103630000AD100F031FC144B03221D608023DB050E
:103640005A629D6200F008FD8023BA681B039A420B
:1036500008D9002E06D000220A4B0C495A621A687B
:103660000A401A600198FEF761F9002005B0F0BD2C
:10367000009A0299D2181278CA540133D4E7C0468E
:103680005443FF1F00C8004000C00040FFFFFEFF82
:10369000F0B587B0029103920400FEF733F9019070
:1036A00000F0FAFB802302250122234EDB05356062
:1036B0005D629A6200F0D0FC204F3B682B42FCD147
:1036C00020230493049B5A1E0492002BFAD11C4D14
:1036D0002B68002BFCDA0120FFF7FCFD002802D04C
:1036E000112007B0F0BD2000039A029900F074FB8E
:1036F000022304003A681A42FCD120230593059B5B
:103700005A1E0592002BFAD12B68002BFCDA0120FF
:10371000FFF7E0FD051EE3D100F0BEFB802303228E
:10372000DB0535605A629D6200F096FC0198FEF759
:10373000FDF8E0B2D5E7C04600C0004090C80040A8
:1037400000C80040F0B5802489B00600FEF7DAF822
:10375000E405A36A02250393029000F09DFB012378
:10376000304F3D606562A36200F076FC2E4C23680A
:103770002B42FCD120230593059B5A1E0592002B5A
:10378000FAD12A4D2B68002BFCDA0120FFF7A2FDAD
:10379000002803D01124200009B0F0BD244B236081
:1037A000022322681A42FCD120230693069B5A1E4C
:1037B0000692002BFAD12B68002BFCDA0120FFF7D0
:1037C00089FD021EE6D11B4B03211E600300019000
:1037D0000090202000F0A8FB022322681A42FCD1AE
:1037E00020230793079B5A1E0792002BFAD12B68C0
:1037F000002BFCDA0320FFF76DFD041ECAD100F098
:103800004BFB80230322DB053C605A629C6200F084
:1038100023FC039B002B01D1FFF776FD0298FEF7F6
:1038200085F8B8E700C0004090C8004000C80040DC
:103830000100000694C8004007B50002019104226F
:10384000000A01A9FFF724FF0EBD000073B50500B3
:1038500005240B4AA3005B429B1819686B46DE1DCA
:103860003000FFF7B3FA022804D133782B55013C1E
:10387000EFD276BD052CFCD00128FAD10230F8E752
:10388000140900111F2807D8012380228340D20584
:1038900091680B43936070473F2808D8012380222A
:1038A00020388340D20551690B435361F3E75F2809
:1038B000F1D80123802240388340D205116A0B439E
:1038C0001362E8E71F2807D8012280218240C9053A
:1038D0008B6893438B6070473F2808D80122802172
:1038E00020388240C9054B6993434B61F3E75F2859
:1038F000F1D80122802140388240C9050B6A9343E8
:103900000B62E8E71F2810D880230200DB05153A78
:103910001968012A06D820229143196019680A43C0
:103920001A60704701228240F6E73F2811D88023B1
:103930000200DB05353AD968032A06D810229143E4
:10394000D960D9680A43DA60EBE701222038824067
:10395000F5E75F28E5D842238022181A413B8340CF
:10396000D205516A99435162516A0B435362D8E7B9
:1039700010B50400012813D1A022184992050B6844
:103980005B015B0913430B60154B164A1968114024
:10399000154A0A431A60402219680A431A6010BD8A
:1039A0000028FCD101000A2000F0EEFA21000B20D3
:1039B00000F0EAFAC0220A4B920019680A4340213B
:1039C0001A601A688A431A60B022044912060B680A
:1039D0005B015B0913430B60E1E7C04614F0004054
:1039E0001CF000407F00FEFF80FD010072B6074A18
:1039F0001368013313600422054B1A600023054A43
:103A000013608022D2055360FEE7C0467808FF1F8E
:103A1000C0F00040C4F0004005490B68002B05D100
:103A2000044A0A6004490A60044A13607047C046A9
:103A3000140AFF1F841E0000380AFF1FC4F0004054
:103A40000023034A1360034A1360034A136070475C
:103A500054F0004040F1004044F10040002310B514
:103A6000184C8AB0009301932378012B27D0694624
:103A7000012000F079FA002817D1009B1249029327
:103A8000019B06AA0393114B02A81B680493104BD9
:103A90001B68059300F0D8F810220E4906A800F024
:103AA00063F8002804D1FF23237000200AB010BD62
:103AB0000123094A074902A8237000F0C5F8012034
:103AC000F4E7C0464464FF1F1029001108290011C3
:103AD0000C290011202900114864FF1F13B501248F
:103AE0006946012000F040FA034B00940193FFF770
:103AF000B5FF200016BDC046BB0B000010B5FFF798
:103B00009FFFFFF7EBFF002802D0024B984710BD44
:103B1000FEE7C046E1A2000002B471464908490030
:103B2000095649008E4402BC7047C04602B4714633
:103B300049084900095C49008E4402BC7047C046F0
:103B400003B47146490840004900095A49008E44AF
:103B500003BC70470000000001B40248844601BC69
:103B6000604700BF01D7000001B40248844601BC91
:103B7000604700BFCD4C010001B40248844601BC3F
:103B8000604700BFC1F7000001B40248844601BC91
:103B9000604700BF53B9000001B40248844601BC2D
:103BA000604700BF8B52010001B40248844601BC4B
:103BB000604700BF6911010001B40248844601BC9E
:103BC000604700BFE927000001B40248844601BCF9
:103BD000604700BF4DF9000001B40248844601BCB3
:103BE000604700BF7997000001B40248844601BCD9
:103BF000604700BFD1AE000001B40248844601BC5A
:103C0000604700BF8D11010001B40248844601BC29
:103C1000604700BF6137010001B40248844601BC1F
:103C2000604700BFBD0B010001B40248844601BCDF
:103C3000604700BFB352010001B40248844601BC92
:103C4000604700BF8552010001B40248844601BCB0
:103C5000604700BFDD3F000001B40248844601BC5C
:103C6000604700BFC56D010001B40248844601BC35
:103C7000604700BF3D71010001B40248844601BCA9
:103C8000604700BFED68010001B40248844601BCF2
:103C9000604700BFD9B0000001B40248844601BCAF
:103CA000604700BFB70E000001B40248844601BC63
:103CB000604700BF7912010001B40248844601BC8C
:103CC000604700BFC9A9000001B40248844601BC96
:103CD000604700BFE512010001B40248844601BC00
:103CE000604700BF0934010001B40248844601BCAA
:103CF000604700BF116E000001B40248844601BC59
:103D0000604700BF9D6A000001B40248844601BCC0
:103D1000604700BFA9D8000001B40248844601BC36
:103D2000604700BF51B8000001B40248844601BC9E
:103D3000604700BFF535010001B40248844601BC6C
:103D4000604700BFEDA5000001B40248844601BCF5
:103D5000604700BF19FA000001B40248844601BC64
:103D6000604700BF090E000001B40248844601BC50
:103D7000604700BF0167010001B40248844601BCEE
:103D8000604700BF0534010001B40248844601BC0D
:103D9000604700BFADAE000001B40248844601BCDC
:103DA000604700BFDD0C010001B40248844601BC3D
:103DB000604700BFC1A5000001B40248844601BCB1
:103DC000604700BFE94C010001B40248844601BCD1
:103DD000604700BF0134010001B40248844601BCC1
:103DE000604700BF9573010001B40248844601BCDE
:103DF000604700BF090E000001B40248844601BCC0
:103E0000604700BF156B010001B40248844601BC45
:103E1000604700BFC166010001B40248844601BC8E
:103E2000604700BF8512010001B40248844601BC0E
:103E3000604700BFF9ED000001B40248844601BCB0
:103E4000604700BF016C010001B40248844601BC18
:103E5000604700BF8944000001B40248844601BCA9
:103E6000604700BFC115010001B40248844601BC8F
:103E7000604700BF75F8000001B40248844601BCE9
:103E8000604700BFE9D4000001B40248844601BC89
:103E9000604700BF0189000001B40248844601BCAC
:103EA000604700BF75A9000001B40248844601BC08
:103EB000604700BF5976010001B40248844601BC46
:103EC000604700BFE9F6000001B40248844601BC27
:103ED000604700BF21A9000001B40248844601BC2C
:103EE000604700BF6DF6000001B40248844601BC83
:103EF000604700BFF1B5001101B40248844601BC1F
:103F0000604700BFED6B010001B40248844601BC6C
:103F1000604700BF6D0B010001B40248844601BC3C
:103F2000604700BF2D6C010001B40248844601BC0B
:103F3000604700BF496D010001B40248844601BCDE
:103F4000604700BFF90D010001B40248844601BC7E
:103F5000604700BF2144000001B40248844601BC10
:103F6000604700BFBD5C010001B40248844601BC4B
:103F7000604700BFE1AC000001B40248844601BCC8
:103F8000604700BFC95C010001B40248844601BC1F
:103F9000604700BF49A2001101B40248844601BC39
:103FA000604700BF71B0000001B40248844601BC04
:103FB000604700BFD544010001B40248844601BCFB
:103FC000604700BF8D82000001B40248844601BCF6
:103FD000604700BFF935010001B40248844601BCC6
:103FE000604700BFE917010001B40248844601BCE4
:103FF000604700BF8914010001B40248844601BC37
:10400000604700BF85C1000001B40248844601BC7E
:10401000604700BFE90B010001B40248844601BCBF
:10402000604700BF0D52010001B40248844601BC44
:10403000604700BF8937010001B40248844601BCD3
:10404000604700BFCD0C010001B40248844601BCAA
:10405000604700BFDD0A010001B40248844601BC8C
:08406000604700BF9DA90000AC
:1040680002000000AABE001101000000B8BC001147
:1040780002000000A6BE001101000000A840FF1FBA
:1040880002000000C0BC001101000000C461FF1F55
:1040980002000000A4BE0011030000003861FF1FE9
:1040A8001200000002000000AABE0011010000007A
:1040B80000BD001102000000A6BE001101000000B2
:1040C800FDBC0011020000000ABD00110300000041
:1040D8007361FF1F02000000A4BE0011030000006E
:1040E8008861FF1F02000000A6BE00110100000049
:1040F800FCBC00110200000008BD00110300000014
:104108004961FF1F02000000A4BE00110300000067
:104118006A61FF1F02000000AABE00110100000032
:1041280044BD001102000000A6BE001101000000FD
:10413800F141FF1F0200000056BD00110100000000
:104148003BBD001102000000A6BE001101000000E6
:10415800F041FF1F0200000054BD001101000000E3
:104168009061FF1F02000000A6BE001101000000C0
:10417800EF41FF1F0200000052BD001101000000C6
:104188002BBD001102000000A6BE001101000000B6
:10419800EE41FF1F0200000050BD001101000000A9
:1041A80026BD001102000000A6BE0011010000009B
:1041B800ED41FF1F020000004EBD0011010000008C
:1041C80021BD001102000000A6BE00110100000080
:1041D800EC41FF1F020000004CBD0011010000006F
:1041E8001CBD0011020202020202000000000000D1
:1041F80016150000BD4B0011834B001198BD00112E
:1042080090011D0018001800FFFF070102030405B4
:104218000602010600000000000000000000000087
:104228000000000000000000000000000000000086
:104238000300000002000000AABE001101000000F7
:10424800B8BD001102000000A6BE00110100000068
:10425800AC42FF1F02000000C2BD001101000000B7
:10426800BE61FF1F02000000A4BE00110300000091
:104278002864FF1F02000000A6BE00110100000014
:10428800AC42FF1F02000000C0BD00110100000089
:10429800C061FF1F02000000A4BE0011030000005F
:1042A8002064FF1F120800000000000000C6C600BE
:1042B80000000000000000001311000000010000D1
:1042C80000000111FFFF00005048593600000000AF
:1042D800000000000B000500F0000000B4000028FA
:1042E800002800283075A000A000A000A000000849
:1042F8000008E001F000100010001000100010008D
:10430800100050005000500010001000D0070000AE
:10431800000000000F0001000500307507001000C4
:10432800010081FF00000000FF000000317400114F
:1043380039720011C96F0011FFFF0100FF00000072
:104348004D9E0011C99B0011E19A00110000000068
:104358000000000000000800040000003B00010805
:104368005902E00188212800FF0000000200000037
:10437800AABE00110100000070BF00110200000079
:10438800A6BE001101000000F143FF1F020000005B
:10439800A2BE0011010000000068FF1F020000001B
:1043A800A6BE001101000000F043FF1F020000003C
:1043B800A0BE001101000000EE43FF1F0200000034
:1043C800A6BE001101000000EC43FF1F0200000020
:1043D8009EBE001101000000E443FF1F18001800F2
:1043E8001D0090010200000302020000020000000C
:1043F800AABE00110100000084BF001102000000E5
:10440800A6BE0011010000003444FF1F0200000096
:104418009CBE001100000000000000000200000027
:0E442800A4BE0011030000002068FF1F20FF4B
:040000051FFF184180
:00000001FF
